:020000020000FC
:100000000C94C63418951895189518951895189548
:100010001895189518951895189518951895189578
:100020001895189518951895189518951895189568
:100030001895189518951895189518951895189558
:100040001895189518951895189518951895189548
:100050000C94B20B18951895189518951895189535
:100060001895189518951895189518951895189528
:100070001895189518951895189518951895189518
:100080001895189518951895189518951895189508
:1000900018951895189518951895189518951895F8
:1000A00018951895189518951895189518951895E8
:1000B00018951895189518951895189518951895D8
:1000C00018951895189518951895189518951895C8
:1000D00018951895189518951895189518951895B8
:1000E00018951895189518951895189518951895A8
:1000F0001895189518951895189518951895189598
:100100001895189518951895189518951895189587
:100110001895189518951895189518950C94A10B85
:100120001895189518951895189518951895189567
:10013000189518950C94020B189518951895189504
:100140001895189518951895189518951895189547
:100150001895189518951895189518951895189537
:100160001895189518951895189518951895189527
:100170001895189518951895189518951895189517
:100180001895189518951895189518951895189507
:1001900018951895189518951895189518951895F7
:1001A00018951895189518951895189518951895E7
:1001B00018951895189518951895189518951895D7
:1001C00018951895189518951895189518951895C7
:1001D00018951895189518951895189518951895B7
:1001E00018951895189518951895189518951895A7
:1001F00018951895189518951895189544241FBCAE
:1002000037CB7ABC26B8A2BD41F61CBE6EBA0DBE75
:10021000FC0C633C5C1D633E6EE3A33E5C1D633ED1
:10022000FC0C633C6EBA0DBE41F61CBE26B8A2BDE6
:1002300037CB7ABC44241FBC93CC6CBD89BC96BD23
:10024000F50AB3BD6D15C9BDA213D7BD45D3573F40
:10025000A213D7BD6D15C9BDF50AB3BD89BC96BD46
:1002600093CC6CBD14BEA1BD6FEDFCBDDC252FBED3
:10027000E9383F3FDC252FBE6FEDFCBD14BEA1BDAC
:100280001F1F1F00000000001C1E1F1F1F1F1F1F1D
:100290001F1F1F1F1F1F1E1C00000000001F1F1F0D
:1002A0001F1F1F1F1F1F0F07070F1F1F1F1F1F1FAE
:1002B00000000000001F1F1F1F1F1F00001F1F1F27
:1002C0000500010403022020052020FF000701048F
:1002D00003060007010603020506FF2020FF0507AD
:1002E000000603020507000403020000012020FFAE
:1002F00005070104030205070103030205070704BC
:100300002020050707040303050701042020001F20
:100310002C3D630001020408102040000306010484
:1003200007020524212A2130210004020136213A46
:07033000213D21412146217E
:100338000000742A10003C246526202768279A2785
:10034800D52711284B289028C52800291329562974
:10035800B929F729382A00002F3210002D306C30C7
:100368007F309430B330DE30283142315731CA31D2
:10037800DB31DE31EF3100321132223200003D3400
:1003880010004B328F32A232B732D032FB324133B7
:100398005B337033D533E633EC33FD330E341F341F
:1003A80030340001933A903A45833A02833A11ED8A
:1003B800390BB239010B3A01833A01833A01833A86
:1003C800020B3A059F3901E03901ED3903BB3902C7
:1003D800ED3903E939FB00E612E23CD103E330D002
:1003E80000E612E237D100E612E234D103E328D066
:1003F80000E713E02FD103E323D000E713E02AD16D
:1004080002E01ED000E713E025D108E019D000E78C
:1004180013E020D101E014D000E612E21BD100E67F
:1004280012E218D106E00CD000E713E013D10CE07B
:1004380007D000E713E00ED100E612E20BD10895D1
:100448008A93802FE4E4F6E000810F7B00830CE2BE
:1004580010E000D100916406007F00936406082F25
:1004680002950F7010916406102B10936406E4E453
:10047800F6E00081006800830CE210E0EBD0E4E4D1
:10048800F6E000810F7700830CED10E0E3D00091D7
:100498006406007F009364068F7000916406082B41
:1004A80000936406E4E4F6E00081006800830CE24F
:1004B80010E0D0D0E4E4F6E000810F7700830CED83
:1004C80010E0C8D0899108958A93802FE4E4F6E07B
:1004D8000081006400830CE210E0BCD00091640647
:1004E800007F00936406082F02950F701091640630
:1004F800102B10936406E4E4F6E0008100680083A2
:100508000CE210E0A7D0E4E4F6E000810F77008366
:100518000CED10E09FD000916406007F0093640604
:100528008F7000916406082B00936406E4E4F6E0FB
:100538000081006800830CE210E08CD0E4E4F6E06F
:1005480000810F7700830CED10E084D08991089525
:100558000E944B38C801A0E007C0B0E0FC01EA0FD8
:10056800FB1F0081B1DFA395B0E0FC01EA0FFB1F80
:100578000081002311F0A13180F3E4E00C945C3891
:100588005FDF07EB15E2E4DF08951BEC10935200E0
:1005980018E010935000E1E5F0E0108113FFFBCF65
:1005A800003221F402EC0093550003C003EC0093E1
:1005B8005500E0E5F0E0008100610083E1E5F0E04E
:1005C800008104FFFBCF08ED04BF04E00093400066
:1005D800E0E5F0E000810E7F0083089500E010E080
:1005E80000930C0210930D0200EB0093010202E24B
:1005F8000093020203E00093040203E00093200248
:1006080008E200932102E0E0F2E00081016000834B
:10061800089501E00093280200E300932902089559
:1006280001E00093300208E30093310208950DE0E1
:100638000093200300E40093210300E000932203C9
:1006480000E50093240300EE0093280300EE0093D6
:100658002A0308950150104098018901232BD1F7EE
:1006680008958A93802F04C008EE1DEF0E94561348
:100678008A95082F802F0023B9F7899108950E9441
:100688004A3880E090E0A0E0B0E04EE0442E1BC085
:10069800442D50E0440F551F440F551FFA01ED53E8
:1006A800FA4D0080118022803380442D50E0440FA1
:1006B800551F440F551FFA01E953FA4D0082118264
:1006C800228233824A9441E0441610F7E7ECF5E2BF
:1006D8000083118322833383442423C0042D10E034
:1006E800000F111F000F111FF801E450FE4F459134
:1006F800559165917491042D10E0000F111F000FA2
:10070800111FF801E953FA4D0081118122813381CB
:100718000E94CF36AC01BD010E946E36C801D901D6
:1007280043940FE04016D0F28C019D01E5E00C9453
:100738005B380E944A3880E090E0A0E0B0E04EE0EC
:10074800442E1BC0442D50E0440F551F440F551F25
:10075800FA01E150FA4D0080118022803380442D47
:1007680050E0440F551F440F551FFA01ED5FF94D36
:1007780000821182228233824A9441E0441610F7A3
:10078800E3E0F6E20083118322833383442423C009
:10079800042D10E0000F111F000F111FF801E45085
:1007A800FE4F4591559165917491042D10E0000F0D
:1007B800111F000F111FF801ED5FF94D0081118124
:1007C800228133810E94CF36AC01BD010E946E3672
:1007D800C801D90143940FE04016D0F28C019D0165
:1007E800E5E00C945B380E944A3880E090E0A0E095
:1007F800B0E04EE0442E1BC0442D50E0440F551F7E
:10080800440F551FFA01E55CF94D008011802280E4
:100818003380442D50E0440F551F440F551FFA01F3
:10082800E15CF94D00821182228233824A9441E0D0
:10083800441610F7EFE3F6E2008311832283338333
:10084800442423C0042D10E0000F111F000F111FB6
:10085800F801E450FE4F4591559165917491042D2E
:1008680010E0000F111F000F111FF801E15CF94D96
:1008780000811181228133810E94CF36AC01BD01F4
:100888000E946E36C801D90143940FE04016D0F299
:100898008C019D01E5E00C945B380E944A3880E0A9
:1008A80090E0A0E0B0E04EE0442E1BC0442D50E0A4
:1008B800440F551F440F551FFA01E958F94D0080A0
:1008C800118022803380442D50E0440F551F440F7F
:1008D800551FFA01E558F94D0082118222823382B0
:1008E8004A9441E0441610F7EBE7F6E200831183DF
:1008F80022833383442423C0042D10E0000F111FEA
:10090800000F111FF801E450FE4F45915591659174
:100918007491042D10E0000F111F000F111FF80132
:10092800E558F94D00811181228133810E94CF362B
:10093800AC01BD010E946E36C801D90143940FE095
:100948004016D0F28C019D01E5E00C945B380E94C2
:100958004A3880E090E0A0E0B0E04EE0442E1BC0B2
:10096800442D50E0440F551F440F551FFA01ED5414
:10097800F94D0080118022803380442D50E0440FCF
:10098800551F440F551FFA01E954F94D0082118291
:10099800228233824A9441E0441610F7E7EBF6E2EC
:1009A8000083118322833383442423C0042D10E061
:1009B800000F111F000F111FF801E450FE4F459161
:1009C800559165917491042D10E0000F111F000FCF
:1009D800111FF801E954F94D0081118122813381F9
:1009E8000E94CF36AC01BD010E946E36C801D90104
:1009F80043940FE04016D0F28C019D01E5E00C9481
:100A08005B380E944A3880E090E0A0E0B0E04EE019
:100A1800442E1BC0442D50E0440F551F440F551F52
:100A2800FA01E151F94D0080118022803380442D74
:100A380050E0440F551F440F551FFA01ED50F94D72
:100A480000821182228233824A9441E0441610F7D0
:100A5800E3EFF6E20083118322833383442423C027
:100A6800042D10E0000F111F000F111FF801E450B2
:100A7800FE4F4591559165917491042D10E0000F3A
:100A8800111F000F111FF801ED50F94D0081118160
:100A9800228133810E94CF36AC01BD010E946E369F
:100AA800C801D90143940FE04016D0F28C019D0192
:100AB800E5E00C945B380E944A3880E090E0A0E0C2
:100AC800B0E04AE0442E1BC0442D50E0440F551FAF
:100AD800440F551FFA01E55DF84D00801180228012
:100AE8003380442D50E0440F551F440F551FFA0121
:100AF800E15DF84D00821182228233824A9441E0FE
:100B0800441610F7EFE2F7E2008311832283338360
:100B1800442423C0042D10E0000F111F000F111FE3
:100B2800F801E85CFD4F4591559165917491042D4C
:100B380010E0000F111F000F111FF801E15DF84DC3
:100B480000811181228133810E94CF36AC01BD0121
:100B58000E946E36C801D90143940BE04016D0F2CA
:100B68008C019D01E5E00C945B380E944A3880E0D6
:100B780090E0A0E0B0E04AE0442E1BC0442D50E0D5
:100B8800440F551F440F551FFA01E95AF84D0080CC
:100B9800118022803380442D50E0440F551F440FAC
:100BA800551FFA01E55AF84D0082118222823382DC
:100BB8004A9441E0441610F7EBE5F7E2008311830D
:100BC80022833383442423C0042D10E0000F111F17
:100BD800000F111FF801E85CFD4F45915591659193
:100BE8007491042D10E0000F111F000F111FF80160
:100BF800E55AF84D00811181228133810E94CF3658
:100C0800AC01BD010E946E36C801D90143940BE0C6
:100C18004016D0F28C019D01E5E00C945B380E94EF
:100C28004A3880E090E0A0E0B0E04AE0442E1BC0E3
:100C3800442D50E0440F551F440F551FFA01ED573E
:100C4800F84D0080118022803380442D50E0440FFD
:100C5800551F440F551FFA01E957F84D00821182BC
:100C6800228233824A9441E0441610F7E7E8F7E21B
:100C78000083118322833383442423C0042D10E08E
:100C8800000F111F000F111FF801E85CFD4F45917F
:100C9800559165917491042D10E0000F111F000FFC
:100CA800111FF801E957F84D008111812281338124
:100CB8000E94CF36AC01BD010E946E36C801D90131
:100CC80043940BE04016D0F28C019D01E5E00C94B2
:100CD8005B380E944A3880E090E0A0E0B0E04AE04B
:100CE800442E1BC0442D50E0440F551F440F551F80
:100CF800FA01E155F84D0080118022803380442D9F
:100D080050E0440F551F440F551FFA01ED54F84D9C
:100D180000821182228233824A9441E0441610F7FD
:100D2800E3EBF7E20083118322833383442423C057
:100D3800042D10E0000F111F000F111FF801E85CCF
:100D4800FD4F4591559165917491042D10E0000F68
:100D5800111F000F111FF801ED54F84D008111818A
:100D6800228133810E94CF36AC01BD010E946E36CC
:100D7800C801D90143940BE04016D0F28C019D01C3
:100D8800E5E00C945B380E944A3880E090E0A0E0EF
:100D9800B0E04AE0442E1BC0442D50E0440F551FDC
:100DA800440F551FFA01E552F84D0080118022804A
:100DB8003380442D50E0440F551F440F551FFA014E
:100DC800E152F84D00821182228233824A9441E036
:100DD800441610F7EFEDF7E2008311832283338383
:100DE800442423C0042D10E0000F111F000F111F11
:100DF800F801E85CFD4F4591559165917491042D7A
:100E080010E0000F111F000F111FF801E152F84DFB
:100E180000811181228133810E94CF36AC01BD014E
:100E28000E946E36C801D90143940BE04016D0F2F7
:100E38008C019D01E5E00C945B380E944A3880E003
:100E480090E0A0E0B0E04AE0442E1BC0442D50E002
:100E5800440F551F440F551FFA01E95FF74D0080F5
:100E6800118022803380442D50E0440F551F440FD9
:100E7800551FFA01E55FF74D008211822282338205
:100E88004A9441E0441610F7EBE0F8E2008311833E
:100E980022833383442423C0042D10E0000F111F44
:100EA800000F111FF801E85CFD4F459155916591C0
:100EB8007491042D10E0000F111F000F111FF8018D
:100EC800E55FF74D00811181228133810E94CF3681
:100ED800AC01BD010E946E36C801D90143940BE0F4
:100EE8004016D0F28C019D01E5E00C945B380E941D
:100EF8004A3880E090E0A0E0B0E046E0442E1BC015
:100F0800442D50E0440F551F440F551FFA01ED5C66
:100F1800F74D0080118022803380442D50E0440F2B
:100F2800551F440F551FFA01E95CF74D00821182E5
:100F3800228233824A9441E0441610F7E7E3F8E24C
:100F48000083118322833383442423C0042D10E0BB
:100F5800000F111F000F111FF801EC59FD4F4591AB
:100F6800559165917491042D10E0000F111F000F29
:100F7800111FF801E95CF74D00811181228133814D
:100F88000E94CF36AC01BD010E946E36C801D9015E
:100F9800439407E04016D0F28C019D01E5E00C94E3
:100FA8005B380E944A3880E090E0A0E0B0E046E07C
:100FB800442E1BC0442D50E0440F551F440F551FAD
:100FC800FA01E15BF74D0080118022803380442DC7
:100FD80050E0440F551F440F551FFA01ED5AF74DC5
:100FE80000821182228233824A9441E0441610F72B
:100FF800E3E5F8E20083118322833383442423C08A
:10100800042D10E0000F111F000F111FF801EC59FB
:10101800FD4F4591559165917491042D10E0000F95
:10102800111F000F111FF801ED5AF74D00811181B2
:10103800228133810E94CF36AC01BD010E946E36F9
:10104800C801D901439407E04016D0F28C019D01F4
:10105800E5E00C945B380E944A3880E090E0A0E01C
:10106800B0E046E0442E1BC0442D50E0440F551F0D
:10107800440F551FFA01E559F74D00801180228071
:101088003380442D50E0440F551F440F551FFA017B
:10109800E159F74D00821182228233824A9441E05D
:1010A800441610F7EFE6F8E20083118322833383B6
:1010B800442423C0042D10E0000F111F000F111F3E
:1010C800F801EC59FD4F4591559165917491042DA6
:1010D80010E0000F111F000F111FF801E159F74D23
:1010E80000811181228133810E94CF36AC01BD017C
:1010F8000E946E36C801D901439407E04016D0F229
:101108008C019D01E5E00C945B380E944A3880E030
:1011180090E0A0E0B0E046E0442E1BC0442D50E033
:10112800440F551F440F551FFA01E957F74D00802A
:10113800118022803380442D50E0440F551F440F06
:10114800551FFA01E557F74D00821182228233823A
:101158004A9441E0441610F7EBE8F8E20083118363
:1011680022833383442423C0042D10E0000F111F71
:10117800000F111FF801EC59FD4F459155916591EC
:101188007491042D10E0000F111F000F111FF801BA
:10119800E557F74D00811181228133810E94CF36B6
:1011A800AC01BD010E946E36C801D901439407E025
:1011B8004016D0F28C019D01E5E00C945B380E944A
:1011C8004A3880E090E0A0E0B0E046E0442E1BC042
:1011D800442D50E0440F551F440F551FFA01ED559B
:1011E800F74D0080118022803380442D50E0440F59
:1011F800551F440F551FFA01E955F74D008211821A
:10120800228233824A9441E0441610F7E7EAF8E272
:101218000083118322833383442423C0042D10E0E8
:10122800000F111F000F111FF801EC59FD4F4591D8
:10123800559165917491042D10E0000F111F000F56
:10124800111FF801E955F74D008111812281338181
:101258000E94CF36AC01BD010E946E36C801D9018B
:10126800439407E04016D0F28C019D01E5E00C9410
:101278005B380E944A3880E090E0A0E0B0E046E0A9
:10128800442E1BC0442D50E0440F551F440F551FDA
:10129800FA01E154F74D0080118022803380442DFB
:1012A80050E0440F551F440F551FFA01ED53F74DF9
:1012B80000821182228233824A9441E0441610F758
:1012C800E3ECF8E20083118322833383442423C0B0
:1012D800042D10E0000F111F000F111FF801EC5929
:1012E800FD4F4591559165917491042D10E0000FC3
:1012F800111F000F111FF801ED53F74D00811181E7
:10130800228133810E94CF36AC01BD010E946E3626
:10131800C801D901439407E04016D0F28C019D0121
:10132800E5E00C945B380E944738842FA52F0E9473
:101338000F36482F50E0440F551F440F551FFA0130
:10134800E152F74D40815181628173810E94B2362A
:10135800280139010A2F10E020E030E00E941A36F7
:10136800A801B901820193010E944837482F50E033
:10137800440F551F440F551FFA01E152F74D4081A4
:101388005181628173810E946E3690E0880F991FA7
:10139800880F991FFC01E152F74D008311832283C6
:1013A8003383E8E00C9458380E944738842FA52FDF
:1013B8000E940F36482F50E0440F551F440F551F09
:1013C800FA01E150F74D40815181628173810E9499
:1013D800B236280139010A2F10E020E030E00E94DF
:1013E8001A36A801B901820193010E944837482F93
:1013F80050E0440F551F440F551FFA01E150F74DB7
:1014080040815181628173810E946E3690E0880F1D
:10141800991F880F991FFC01E150F74D0083118334
:1014280022833383E8E00C9458381091480001E097
:10143800009348002091A0003091A2000091A200E2
:101448000C7F04600093A2004FB77894E8E4F0E0C2
:101458000081016000835091CD01EF93FF930F93BA
:101468002F93EBECF1E008ED21E004BF20832F91EE
:101478000F91FF91EF9103E00093CD0188951093B0
:1014880048002093A0003093A2005093CD014FBF95
:101498000895EFECF1E0008107FDFBCF0895F9DF37
:1014A800EFECF1E0008101FF11C006E30093CA01EF
:1014B800EF93FF930F932F93EBECF1E008ED21E00E
:1014C80004BF20832F910F91FF91EF9108959A9374
:1014D8008A93C801DEDFFC01E05CF140F09750F42C
:1014E80040919B2B50E009E010E00E941435800FDA
:1014F800911F17C0803C01E0900798F440919A2B07
:1015080050E00DE110E00E941435980140919B2BAA
:1015180050E007E510E00E941435200F311F820FBC
:10152800931F082F0093C001892F8F718093C101E9
:1015380000E00093C20106E00093CA01EF93FF9315
:101548000F932F93EBECF1E008ED21E004BF20832B
:101558002F910F91FF91EF910091C4018991999179
:1015680008950E944C38C801A22F00E00093060994
:1015780000E000934608FC01E05CF140F09750F46D
:1015880040919B2B50E009E010E00E941435800F39
:10159800911F17C0803C01E0900798F440919A2B66
:1015A80050E00DE110E00E941435980140919B2B0A
:1015B80050E007E510E00E941435200F311F820F1C
:1015C800931F6DDF03E30093CA01082F0093C00146
:1015D800892F8F718093C10100E00093C201A0930D
:1015E800C40105E30093CA0120DF03E00093060964
:1015F80001E000934608E3E00C945D389A938A93DF
:10160800FA93EA930A927A936A935A934A933A938B
:101618002A931A930A930FB6E0E0F2E0008104607F
:1016280000830091612B039507700093612B009153
:10163800602B03950093602B0330B9F400E000930E
:10164800602B0091622B039507700093622B009129
:10165800622B10E0000F111FF801E15DF64D0081CB
:10166800118100933A0310933B030091662B0023EA
:1016780009F454C000917F2A1091802A212F220F4B
:10168800220B322F4091612B50E0440F551F440F1D
:10169800551FFA01E15EF54D4081518162817381E8
:1016A800400F511F621F731F4083518362837383EE
:1016B80000917F2A1091802A212F220F220B322F8E
:1016C8004091622B50E0440F551F440F551FFA01FB
:1016D800E150F64D4081518162817381400F511F65
:1016E800621F731F408351836283738380919B2A97
:1016F80090919C2A019680939B2A90939C2A009112
:101708009D2A10919E2A8017910741F400E00093CA
:10171800662B10E000939B2A10939C2A0FBE099118
:101728001991299139914991599169917991099022
:10173800E991F9918991999118952A931A930A93A5
:101748002FB7009110021091110200937F2A109375
:10175800802A2FBF09911991299118955A924A9276
:10176800BA93AA939A938A93FA93EA933A922A920B
:101778001A920A927A936A935A934A933A932A93BB
:101788001A930A935FB60091662B002309F074C779
:10179800E5EAFAE2008111810F5F1F4F0083118390
:1017A8000091742B0E5F00937F2B80E03BC050911B
:1017B8007F2B5395482F642F082F10E0000F111F1F
:1017C800000F111FF801E150F64D008111812281AF
:1017D800338142E07091842B471B0E948235462F4B
:1017E800A2DD0E941C36482F50E0440F551F440FBD
:1017F800551FFA01E15CF54D008311832283338381
:1018080000E010E020E030E0482F50E0440F551F82
:10181800440F551FFA01E150F64D008311832283CE
:1018280033838395883018F280E03AC050917F2B3B
:10183800482F642F082F10E0000F111F000F111FF1
:10184800F801E15EF54D008111812281338143E089
:101858007091842B471B0E948235462FA5DD0E947C
:101868001C36482F50E0440F551F440F551FFA01EE
:10187800E15AF54D008311832283338300E010E0A1
:1018880020E030E0482F50E0440F551F440F551F0B
:10189800FA01E15EF54D008311832283338383953A
:1018A800883020F20FEF0093662B00E010E020E074
:1018B80030E0EFEAFAE20083118322833383EBEA14
:1018C800FAE20083118322833383E7EAFAE2008392
:1018D80011832283338344249DC0E7EAFAE200811E
:1018E8001181228133810E940F36C801D901042D4C
:1018F80010E0000F111F000F111FF801E15CF54DFA
:1019080000811181228133810E940F36442D50E0DD
:10191800440F551F440F551FFA01E15CF64D4081F5
:101928005181628173810E94CF36AC01BD010E9452
:101938006E360E941C36E7EAFAE20083118322839E
:101948003383EBEAFAE200811181228133810E941C
:101958000F36C801D901042D10E0000F111F000F28
:10196800111FF801E15CF54D00811181228133815D
:101978000E940F36442D50E0440F551F440F551F49
:10198800FA01E15AF64D40815181628173810E94CA
:10199800CF36AC01BD010E946E360E941C36EBEAC0
:1019A800FAE20083118322833383EFEAFAE20081AB
:1019B8001181228133810E940F36C801D901042D7B
:1019C80010E0000F111F000F111FF801E15CF54D29
:1019D80000811181228133810E940F36442D50E00D
:1019E800440F551F440F551FFA01E158F64D408129
:1019F8005181628173810E94CF36AC01BD010E9482
:101A08006E360E941C36EFEAFAE2008311832283C5
:101A18003383439408E0401608F45FCFE7EAFAE21C
:101A28000081118122813381EBEBFAE2008311837B
:101A380022833383EBEAFAE2008111812281338128
:101A4800EFEBFAE20083118322833383EFEAFAE2B1
:101A58000081118122813381E7ECFAE2008311834E
:101A680022833383E3EDFAE20081118122813381FD
:101A7800E7ECFAE24081518162817381041715070E
:101A8800260737077CF4E3EDFAE200811181228111
:101A980033810F5F1F4F2F4F3F4F008311832283E6
:101AA80033830EC0E3EDFAE2008111812281338194
:101AB800015010402040304000831183228333833B
:101AC800EFECFAE20081118122813381EBEBFAE23B
:101AD80040815181628173810417150726073707F2
:101AE8007CF4EFECFAE200811181228133810F5FEF
:101AF8001F4F2F4F3F4F00831183228333830EC024
:101B0800EFECFAE20081118122813381015010400B
:101B1800204030400083118322833383EBECFAE2C8
:101B28000081118122813381EFEBFAE240815181FA
:101B38006281738104171507260737077CF4EBECDD
:101B4800FAE200811181228133810F5F1F4F2F4FED
:101B58003F4F00831183228333830EC0EBECFAE2FC
:101B68000081118122813381015010402040304092
:101B780000831183228333830091652B002321F195
:101B8800EBEBFAE20081118122813381EFECFAE27A
:101B98000083118322833383EFEBFAE20081118102
:101BA80022813381EBECFAE20083118322833383B1
:101BB800E7ECFAE20081118122813381E3EDFAE258
:101BC8000083118322833383EFECFAE200811181D1
:101BD80022813381EBEBFAE240815181628173818A
:101BE800401B510B620B730B4083518362837383D9
:101BF800EBECFAE20081118122813381EFEBFAE20A
:101C08004081518162817381401B510B620B730BC0
:101C18004083518362837383E3EDFAE2008111818B
:101C280022813381E7ECFAE240815181628173813C
:101C3800401B510B620B730B408351836283738388
:101C48000091702B013009F0ADC000917D2B01305F
:101C5800B9F5EBEBFAE200811181228133810E9410
:101C68000F360E9443030E941C36E7E2FBE2008322
:101C7800118322833383EFEBFAE200811181228101
:101C880033810E940F360E949D030E941C36EBE2AE
:101C9800FBE20083118322833383E7ECFAE20081BD
:101CA8001181228133810E940F360E94F7030E941E
:101CB8001C36E3E2FBE2008311832283338396C060
:101CC80000917D2B0230B9F5EBEBFAE2008111812E
:101CD800228133810E940F360E945F050E941C36C4
:101CE800E7E2FBE20083118322833383EFEBFAE21E
:101CF80000811181228133810E940F360E94B9052B
:101D08000E941C36EBE2FBE20083118322833383BB
:101D1800E7ECFAE200811181228133810E940F36BB
:101D28000E9413060E941C36E3E2FBE20083118343
:101D3800228333835BC0EBEBFAE2008111812281BD
:101D480033810E940F360E947B070E941C36E7E20F
:101D5800FBE20083118322833383EFEBFAE20081F5
:101D68001181228133810E940F360E94D5070E947B
:101D78001C36EBE2FBE20083118322833383E7EC1A
:101D8800FAE200811181228133810E940F360E947C
:101D98002F080E941C36E3E2FBE2008311832283B2
:101DA800338324C0EBEBFAE2008111812281338175
:101DB800E7E2FBE20083118322833383EFEBFAE24D
:101DC8000081118122813381EBE2FBE200831183E0
:101DD80022833383E7ECFAE2008111812281338187
:101DE800E3E2FBE20083118322833383E7E2FBE231
:101DF8000081118122813381E3E3FBE2408151813B
:101E080062817381400F511F621F731F408351838A
:101E180062837383EBE2FBE20081118122813381CB
:101E2800E7E3FBE24081518162817381400F511FDA
:101E3800621F731F4083518362837383E3E2FBE273
:101E48000081118122813381EFE2FBE240815181DF
:101E580062817381400F511F621F731F408351833A
:101E6800628373832091872B23952093872B00917E
:101E7800832B10E0F801E75DFC4F0491201708F46C
:101E880045C000E00093872BE3E3FBE2008111816A
:101E980022813381E3EBFAE20083118322833383C7
:101EA80000E010E020E030E0E3E3FBE20083118390
:101EB80022833383E7E3FBE20081118122813381AE
:101EC800E7EBFAE2008311832283338300E010E01A
:101ED80020E030E0E7E3FBE20083118322833383D1
:101EE800EFE2FBE20081118122813381E3ECFAE227
:101EF800008311832283338300E010E020E030E088
:101F0800EFE2FBE2008311832283338300E010E0D9
:101F180020E030E0EFEAFAE2008311832283338382
:101F2800EBEAFAE20083118322833383E7EAFAE2D9
:101F3800008311832283338300E010E020E030E047
:101F4800E6E9FBE200831183228333834424C9C07A
:101F5800042D10E0000F111F000F111FF801E15AA6
:101F6800F54D4081518162817381042D10E0000F8D
:101F7800111F000F111FF801E15AF54D0081118161
:101F8800228133810E945A350E940F36E6E9FBE22E
:101F980040815181628173810E946E36E6E9FBE2DD
:101FA8000083118322833383E7EAFAE200811181F7
:101FB800228133810E940F36C801D901042D10E017
:101FC800000F111F000F111FF801E15AF54D008194
:101FD8001181228133810E940F36442D50E0440F35
:101FE800551F440F551FFA01E156F64D40815181A6
:101FF800628173810E94CF36AC01BD010E946E36AA
:102008000E941C36E7EAFAE20083118322833383B5
:10201800EBEAFAE200811181228133810E940F36B6
:10202800C801D901042D10E0000F111F000F111F66
:10203800F801E15AF54D00811181228133810E9416
:102048000F36442D50E0440F551F440F551FFA0119
:10205800E154F64D40815181628173810E94CF36EF
:10206800AC01BD010E946E360E941C36EBEAFAE212
:102078000083118322833383EFEAFAE2008111811E
:10208800228133810E940F36C801D901042D10E046
:10209800000F111F000F111FF801E15AF54D0081C3
:1020A8001181228133810E940F36442D50E0440F64
:1020B800551F440F551FFA01E152F64D40815181D9
:1020C800628173810E94CF36AC01BD010E946E36D9
:1020D8000E941C36EFEAFAE20083118322833383DD
:1020E800439408E0401608F433CF40E050E060E045
:1020F80071E4E6E9FBE200811181228133810E94CB
:1021080048370E94B33CE6E9FBE20083118322834F
:1021180033830091A12A1091A22A20E030E00E9486
:102128001A36A801B901E6E9FBE200811181228192
:1021380033810E9448370E941C360093992A1093D5
:102148009A2A0091802B10E0F801ED5EFC4F449133
:1021580050E00091992A10919A2A0E942E350093F6
:10216800992A10939A2A0091842B023051F40091F5
:10217800992A10919A2A169507950093992A1093EF
:102188009A2AE7EAFAE20081118122813381EFED90
:10219800FAE20083118322833383EBEAFAE20081B7
:1021A800118122813381E3EEFAE2008311832283D5
:1021B8003383EFEAFAE20081118122813381EBEE69
:1021C800FAE20083118322833383E7EFFAE2008186
:1021D800118122813381EBEEFAE2408151816281E3
:1021E800738104171507260737077CF4E7EFFAE22F
:1021F80000811181228133810F5F1F4F2F4F3F4F85
:1022080000831183228333830EC0E7EFFAE2008153
:1022180011812281338101501040204030400083D9
:10222800118322833383E3EFFAE200811181228153
:102238003381EFEDFAE240815181628173810417A5
:102248001507260737077CF4E3EFFAE200811181CE
:10225800228133810F5F1F4F2F4F3F4F0083118320
:10226800228333830EC0E3EFFAE2008111812281D9
:102278003381015010402040304000831183228375
:102288003383EBECFAE20081118122813381E3EEA2
:10229800FAE240815181628173810417150726078C
:1022A80037077CF4EFEEFAE2008111812281338155
:1022B8000F5F1F4F2F4F3F4F0083118322833383BC
:1022C8000EC0EFEEFAE200811181228133810150C4
:1022D80010402040304000831183228333830091D3
:1022E800652B002339F100E00093652BEFEDFAE24E
:1022F8000081118122813381E3EFFAE200831183A7
:1023080022833383E3EEFAE2008111812281338153
:10231800EFEEFAE20083118322833383EBEEFAE2D5
:102328000081118122813381E7EFFAE20083118372
:1023380022833383E3EFFAE2008111812281338122
:10234800EFEDFAE24081518162817381401B510BAC
:10235800620B730B4083518362837383EFEEFAE25F
:102368000081118122813381E3EEFAE240815181BB
:1023780062817381401B510B620B730B4083518345
:1023880062837383E7EFFAE200811181228133814E
:10239800EBEEFAE24081518162817381401B510B5F
:1023A800620B730B40835183628373830091702B9C
:1023B800013009F0ADC000917D2B0130B9F5EFED8A
:1023C800FAE200811181228133810E940F360E9436
:1023D80051040E941C36EFE3FBE200831183228341
:1023E8003383E3EEFAE200811181228133810E9476
:1023F8000F360E94AB040E941C36E3E4FBE2008324
:10240800118322833383EBEEFAE20081118122816A
:1024180033810E940F360E9405050E941C36EBE3AB
:10242800FBE2008311832283338396C000917D2BC6
:102438000230B9F5EFEDFAE2008111812281338192
:102448000E940F360E946D060E941C36EFE3FBE2E5
:102458000083118322833383E3EEFAE20081118142
:10246800228133810E940F360E94C7060E941C36C3
:10247800E3E4FBE20083118322833383EBEEFAE289
:1024880000811181228133810E940F360E94210729
:102498000E941C36EBE3FBE2008311832283338323
:1024A8005BC0EFEDFAE200811181228133810E9445
:1024B8000F360E9489080E941C36EFE3FBE2008376
:1024C800118322833383E3EEFAE2008111812281B2
:1024D80033810E940F360E94E3080E941C36E3E411
:1024E800FBE20083118322833383EBEEFAE200815F
:1024F8001181228133810E940F360E943D090E947A
:102508001C36EBE3FBE2008311832283338324C070
:10251800EFEDFAE20081118122813381EFE3FBE2E2
:102528000083118322833383E3EEFAE20081118171
:1025380022813381E3E4FBE2008311832283338326
:10254800EBEEFAE20081118122813381EBE3FBE2B9
:102558000083118322833383EFE3FBE2008111813F
:1025680022813381EBE4FBE24081518162817381F6
:10257800400F511F621F731F40835183628373830F
:10258800E3E4FBE20081118122813381EFE4FBE285
:102598004081518162817381400F511F621F731FF7
:1025A8004083518362837383EBE3FBE200811181F3
:1025B80022813381E7E4FBE24081518162817381AA
:1025C800400F511F621F731F4083518362837383BF
:1025D8002091882B23952093882B0091832B10E042
:1025E800F801E75DFC4F0491201708F445C000E0AE
:1025F8000093882BEBE4FBE2008111812281338177
:10260800E7EDFAE2008311832283338300E010E0D0
:1026180020E030E0EBE4FBE2008311832283338384
:10262800EFE4FBE20081118122813381EBEDFAE2D4
:10263800008311832283338300E010E020E030E040
:10264800EFE4FBE20083118322833383E7E4FBE2B8
:102658000081118122813381E7EEFAE20083118340
:102668002283338300E010E020E030E0E7E4FBE27F
:1026780000831183228333835FBE099119912991C5
:1026880039914991599169917991099019902990B5
:102698003990E991F99189919991A991B9914990C4
:1026A800599018959C01C8010197FC01CF01EF2BA7
:1026B800D9F716950795C8010197FC01CF01EF2BB3
:1026C800D9F7C90108950E944B3800E40E942402FA
:1026D800AFEF80E002C0A69583958830A8F4BA2FA2
:1026E80090E005C000E00E946802B6959395983086
:1026F80090F7BB2311F001E001C000E0002391F73F
:102708000FE10E946802F1CFE4E00C945C389A93E0
:102718008A9300E40E94240280E008C090E0FC0153
:10272800E058FD4F04910E94680283958034B0F30D
:102738008991999108950E944B38D80180E090E0E2
:102748002AC00DE210E0AC010E941435F801EA0F2E
:10275800FB1FE83601E0F00714F0E856F1408F015E
:10276800212F220F220B322F0E940F3645E35AEFFA
:102778006EE87CE30E94CF360E94C234AC01440F5D
:10278800551F440F551FFA01E158F64D0083118378
:10279800228333830196883000E0900794F2E4E0C6
:1027A8000C945C380E944B38D80180E090E02AC035
:1027B8000DE210E0AC010E941435F801EA0FFB1F8E
:1027C800E83601E0F00714F0E856F1408F01212FB8
:1027D800220F220B322F0E940F3645E35AEF6EE884
:1027E8007CE30E94CF360E94E53BAC01440F551FA5
:1027F800440F551FFA01E15CF64D008311832283D3
:1028080033830196883000E0900794F2E4E00C945A
:102818005C380E944B38D80180E090E02AC00DE275
:1028280010E0AC010E941435F801EA0FFB1FE836EE
:1028380001E0F00714F0E856F1408F01212F220F34
:10284800220B322F0E940F3645E35AEF6EE87CE3E5
:102858000E94CF360E94C234AC01440F551F440F6A
:10286800551FFA01E15AF64D008311832283338301
:102878000196883000E0900794F2E4E00C945C380C
:102888000E944B38D80180E090E02AC00DE210E0A9
:10289800AC010E941435F801EA0FFB1FE83601E08D
:1028A800F00714F0E856F1408F01212F220F220B78
:1028B800322F0E940F3645E35AEF6EE87CE30E9400
:1028C800CF360E94C234AC01440F551F440F551F28
:1028D800FA01E152F64D0083118322833383019676
:1028E800883000E0900794F2E4E00C945C380E9491
:1028F8004B38D80180E090E02AC00DE210E0AC012E
:102908000E941435F801EA0FFB1FE83601E0F007D2
:1029180014F0E856F1408F01212F220F220B322F9D
:102928000E940F3645E35AEF6EE87CE30E94CF36EB
:102938000E94E53BAC01440F551F440F551FFA0197
:10294800E156F64D00831183228333830196883044
:1029580000E0900794F2E4E00C945C380E944B3855
:10296800D80180E090E02AC00DE210E0AC010E949E
:102978001435F801EA0FFB1FE83601E0F00714F000
:10298800E856F1408F01212F220F220B322F0E948F
:102998000F3645E35AEF6EE87CE30E94CF360E947B
:1029A800C234AC01440F551F440F551FFA01E154BE
:1029B800F64D00831183228333830196883000E02B
:1029C800900794F2E4E00C945C380E9443382801A4
:1029D800662476C0062D10E020E030E00E941A360A
:1029E8004BED5FE069E47FE30E94CF360E94E53B50
:1029F800C801D9018201212F220F220B322F0E94F8
:102A08000F36AC01BD010E94CF36C801D901820141
:102A1800212F220F220B322F0E940F36AC01BD014D
:102A28000E946E3640E050E060E470E40E9448374F
:102A3800480159018201212F220F220B322F0E94B7
:102A48000F36C801D9017724F301E55EFC4F0491E4
:102A580010E020E030E00E941A36080119014BED21
:102A68005FE069E47FE3800191010E94CF360E9414
:102A7800E53BAC01BD010E94CF36C801D9018201F6
:102A8800212F220F220B322F0E940F36AC01BD01DD
:102A98000E946E3640E050E060E87FE30E944837CD
:102AA800A401B5010E946E360E941C36262D30E026
:102AB800220F331FF901E15DF64D00831183639402
:102AC80008E0601608F486CFECE00C9454380E94B5
:102AD800433858014901A0E0B0E080C00DE210E0A1
:102AE800AD010E94143528014A0C5B1C08E640160B
:102AF80001E0500624F008E9400E0EEF501EFD01DB
:102B0800E55EFC4F449150E00DE210E00E94143560
:102B1800C8018A0D9B1D883601E0900714F088567D
:102B280091408201212F220F220B322F0E940F3653
:102B380045E35AEF6EE87CE30E94CF360E94E53BFE
:102B480040E050E060E070E40E9448372801390115
:102B58008C01212F220F220B322F0E940F360801E1
:102B6800190145E35AEF6EE87CE3800191010E9468
:102B7800CF360E94E53B0801190140E050E060E0D3
:102B880070E4800191010E944837A201B3010E94BC
:102B98006E36280139018401212F220F220B322F92
:102BA8000E940F36A201B3010E94CF3628013901D5
:102BB8008401212F220F220B322F0E940F36A201EF
:102BC800B3010E946E360E941C369D01220F331FEE
:102BD800F901E15EF64D008311831196A83000E0FB
:102BE800B0070CF47BCFECE00C9454380E944B38BF
:102BF80020E030E000E010E06ADF69D105E00E94E3
:102C08003503E091992AF0919A2AF39708F4EDC0D8
:102C180080E09CE5A1ECB7E400E010E00093A02B75
:102C28001093A12B08C0E0EAFBE2008111810B5F41
:102C38001F4F008311830091A02B1091A12B083600
:102C480021E012079CF520915D2530915E250091C9
:102C5800A02B1091A12B3BDF02E00E9435030091CD
:102C6800992A10919A2A20E030E00E941A36AC0185
:102C7800BD010E94D137B8F60091992A10919A2A7D
:102C880020E030E00E941A36C801D9010091A02B3B
:102C98001091A12B00939C2B10939D2BE091992AC6
:102CA800F0919A2AB89708F0BECF50C080E09CE512
:102CB800A1ECB7E405E010E0EAD000E010E00093F2
:102CC8005D2510935E2508C0EDE5F5E200811181D0
:102CD800025E1F4F0083118300915D2510915E25D0
:102CE800083E27E0120794F520915D2530915E2576
:102CF80000919C2B10919D2BEADE02E00E94350387
:102D08000091992A10919A2A20E030E00E941A3600
:102D1800AC01BD010E94D137B8F60091992A1091F3
:102D28009A2A20E030E00E941A36C801D9010091A1
:102D38005D2510915E2500939E2B10939F2BE091AB
:102D4800992AF0919A2A749708F0BECFE0919C2BAB
:102D5800F0919D2B349744F0ECE9FBE2008111815E
:102D68000350104000831183E0919E2BF0919F2B1C
:102D78003B9744F0EEE9FBE2008111810A501040D4
:102D88000083118320919E2B30919F2B00919C2BC7
:102D980010919D2B9CDE00919E2B10919F2B0093F0
:102DA8005E2B10935F2B00919C2B10919D2B009311
:102DB8005C2B10935D2B30915D2B232F0EE010E0E0
:102DC8000E94B50A20915C2B0FE010E00E94B50A22
:102DD80030915F2B232F00E110E00E94B50A20916B
:102DE8005E2B01E110E00E94B50A0FEF0093642BFF
:102DF800E4E00C945C3834E03093400930917B2B4C
:102E0800329F00926A0910926B0900936609109329
:102E1800670908950E944B38D801922F24E08D014C
:102E2800EADF00E315E73EDC88E00CC0989F8001EC
:102E380043E00E942835202F8D01DDDF00E41CE9E6
:102E480031DC8A95813090F7E4E00C945C380E947C
:102E58004B38D80122E08D01CEDF08EE1DEF22DCD1
:102E680008EE1DEF1FDC84E090E00AC0282F8D01DA
:102E7800C2DF08EE1DEF16DC08EE1DEF13DC01972C
:102E8800813000E0900794F7E4E00C945C3822E08D
:102E980044E650E00E941435AEDF48E750E0009168
:102EA800852A1091862A0E9446350E94350300E043
:102EB8000093400908958A93812F10E0E8DF00E32A
:102EC80015E7F0DB082F10E0E2DF899108952BE485
:102ED80031E207EB15E20E94983C00E80E94C40228
:102EE80000E310E0D4DF08950E945A3440E050E037
:102EF80064E672E40E94CF360E941C3608950E9450
:102F08004738C801D9012A013B010091852B0023CC
:102F180079F4A201B3018C019D010E945A3440E06A
:102F280050E064E672E40E94CF360E941C3627C047
:102F3800A201B3012A013B010AE010E02091852B90
:102F480030E0021B130B212F220F220B322F0E947D
:102F58000F36A801B901820193010E944837AC01DC
:102F6800BD010E946E36A201B3010E945A3440E0AE
:102F780050E064E672E40E94CF360E941C360B359E
:102F880020E0120714F00BE510E0063A2FEF1207C5
:102F980014F405EA1FEFE8E00C9458380E944B3807
:102FA800A0E0B0E000E00093010204E00E943503D5
:102FB80080E090E019C0E0E0F2E000810860008362
:102FC80000912B020023E1F301E000932B02009112
:102FD800120210911302A00FB11F0091942B1091AF
:102FE800952BA01BB10B0196803A00E090071CF3CB
:102FF80000E10093010200E117E254DBBB2312F465
:10300800A0E0B0E04AE650E08D010E944635E4E0D9
:103018000C945C380E944B3880E090E000E000930C
:10302800010203E00E943503A0E0B0E013C0E0E035
:10303800F2E000810860008300912B020023E1F395
:1030480001E000932B020091120210911302800FED
:10305800911F1196A43600E0B0074CF300E10093ED
:10306800010244E650E08C010E944635E4E00C94ED
:103078005C38E0E0F2E000810061008300913302F7
:103088000023E1F301E0009333024091792B50E0F3
:1030980000911402109115020E942E350895009196
:1030A800542B1091552B7EDB0091542B1091552BEE
:1030B800B0DB0091582B1091592B19DC0091582B3B
:1030C8001091592B4BDC0091542B1091552B0093E8
:1030D800562B1093572B0091562B1091572B2BDB07
:1030E8000091582B1091592B00935A2B10935B2B5E
:1030F80000915A2B10915B2BC3DB08950091542B40
:103108001091552B4FDB0091542B1091552B81DBDF
:103118000091562B1091572B0EDB0091582B1091D4
:10312800592BE5DB0091582B1091592B17DC009196
:103138005A2B10915B2BA4DB4091812B50E00FEFB1
:1031480010E00E94143541DC0091852A1091862AEE
:10315800009326091093270908959A938A9301E00A
:1031680010E00E946B0A902F80E002E010E00E94BD
:103178006B0A10E0802B912B8093852A9093862AE6
:1031880005E010E00E946B0A902F80E006E010E056
:103198000E946B0A10E0802B912B8093542B909304
:1031A800552B07E010E00E946B0A902F80E008E0A2
:1031B80010E00E946B0A10E0802B912B8093562B15
:1031C8009093572B05E110E00E946B0A902F80E046
:1031D80006E110E00E946B0A10E0802B912B80938F
:1031E800582B9093592B07E110E00E946B0A902FFF
:1031F80080E008E110E00E946B0A10E0802B912B20
:1032080080935A2B90935B2B0EE010E00E946B0A80
:10321800902F80E00FE010E00E946B0A10E0802BF6
:10322800912B80935C2B90935D2B00E110E00E9422
:103238006B0A902F80E001E110E00E946B0A10E019
:10324800802B912B80935E2B90935F2B03E010E0F3
:103258000E946B0A0093752B04E010E00E946B0A31
:103268000093762B09EF11E00E946B0A0093782BEC
:1032780007EF11E00E946B0A00937E2B0CE010E030
:103288000E946B0A0093812B0DE010E00E946B0AEC
:1032980000937D2B0BEF11E00E946B0A0093892BA2
:1032A8000CEF11E00E946B0A0093792B06EF11E0F6
:1032B8000E946B0A00937B2B05EF11E00E946B0ABA
:1032C8000093822B0DEF11E00E946B0A00937C2B78
:1032D80002E110E00E946B0A0093802B0AE010E0E4
:1032E8000E946B0A802F90E00BE010E00E946B0AAE
:1032F800102F00E0802B912B80938A2B90938B2B9F
:1033080003E110E00E946B0A0093832B08EF11E0A1
:103318000E946B0A00936A2B0EEF11E00E946B0A61
:103328000093732B04E110E00E946B0A0093742B46
:1033380000E010E00E946B0A0093842B04EF11E078
:103348000E946B0A00936C2B03EF11E00E946B0A3A
:103358000093852B0BE110E00E946B0A0093862BEB
:10336800EAE8FBE200810160008389919991089560
:103378000E944B38D801AB3500E0B00714F0AAE53D
:10338800B0E00091702B002331F00091832B0330C3
:1033980011F088E40DC0BB2312F48CE309C04AE0A5
:1033A80050E08D010E944635102F06E0109F802DB9
:1033B80000E80E94240290E0FC01E054FD4F0491D3
:1033C8000E94680201E80E94240290E0FC01EF5389
:1033D800FD4F04910E94680202E80E94240290E0D6
:1033E800FC01EE53FD4F04910E94680200EC0E941C
:1033F800240290E0FC01ED53FD4F04910E94680205
:1034080001EC0E94240290E0FC01EC53FD4F049172
:103418000E94680202EC0E94240290E0FC01EB5337
:10342800FD4F04910E9468020091702B002331F037
:103438000091832B033011F088E40CC0BB2312F4F5
:1034480082E408C04AE050E08D010E94463506E05B
:10345800409F802D04E80E94240290E0FC01E05483
:10346800FD4F04910E94680205E80E94240290E042
:10347800FC01EF53FD4F04910E94680206E80E9488
:10348800240290E0FC01EE53FD4F04910E94680273
:1034980004EC0E94240290E0FC01ED53FD4F0491DE
:1034A8000E94680205EC0E94240290E0FC01EC53A3
:1034B800FD4F04910E94680206EC0E94240290E0ED
:1034C800FC01EB53FD4F04910E94680203E80E943F
:1034D800240200E20E94680203EC0E94240200E237
:1034E8000E946802E4E00C945C380E944738C801E6
:1034F800EAE8FBE2018107FF02C005E501C008E533
:1035080099230AF473C010E0801791070CF06EC07D
:103518004AE050E08C010E944635402F4A5F0091F6
:103528008A2B10918B2B0E9428350170002309F0FB
:103538005DC00091692B083018F007E00093692BF3
:1035480000917E2B013031F42091692B00E717E1BF
:1035580052DCA0C000917E2B0230D1F4853100E00E
:10356800900734F42091692B00EE1EE244DC92C0EF
:103578008B3400E0900734F02091692B00EA1FE0BB
:103588003ADC88C02091692B00E717E134DC82C05F
:1035980000917E2B0330A9F42091692BA22F0AE019
:1035A800402E55244AE050E08C010E944635401ACE
:1035B800510A00E416E0A2010E9414352A2F1BDCF0
:1035C80069C02091692BA22F0AE0402E55244AE0B9
:1035D80050E08C010E944635401A510A00E416E07A
:1035E800A2010E9414352A2F15DC54C099230AF031
:1035F80047C00091762B10E020E030E00E941A3698
:103608002801390103E010E04091812A5091822A73
:103618000E941435212F220F220B322F0E940F36C1
:103628000E946538A801B901820193010E94D1372F
:1036380038F5A4E04CEE5FEF8C010E944635A01BE4
:103648004A2F00918A2B10918B2B0E9428350170EC
:103658000023B1F442E00091692B0E94F6340093F4
:10366800692B863F0FEF90072CF02091692B00E51E
:1036780016E4C1DB2091692B00E61DE6BCDB0AC01D
:1036880000E010E00093932A1093942A0093872A6D
:103698001093882AE8E00C9458389A938A9380917A
:1036A800852A9091862A0196AC01652F660F660BD4
:1036B800762F00E01CE62CED32E00E94AD3548E0A4
:1036C80050E060E070E00E94AD3548E050E060E016
:1036D80070E00E945A3540E750E060E070E00E94D8
:1036E800AD3500939F2A1093A02A45E000919F2AA8
:1036F8001091A02A0E94223540E250E00E94143521
:1037080000939F2A1093A02A48EC50E000919F2A2A
:103718001091A02A0E942E350093A12A1093A22A64
:1037280000919F2A1091A02A00939D2A10939E2A07
:1037380046E150E00091852A1091862A0E9446357C
:103748000093A32A1093A42A8991999108958A93A2
:103758000091732B10E0F801E25FFC4F0491002305
:1037680059F100916E2B002339F583DC2091732BDE
:1037780030E0F901E25FFC4F249130E002171307B3
:10378800DCF480E017C02CE531E207EB15E20E947B
:10379800983C00E80E94C40208E710E078DB08EED5
:1037A8001DEF0E94561301E00E94240202E00E94CD
:1037B80035038395853038F3899108951091200257
:1037C800137E109320020A95000F000F109120021B
:1037D800102B109320020895C0DC5FDF0E94EF01D8
:1037E8000091822B023039F400916E2B002319F4DA
:1037F8000E948B1302C00E94671320915E2B3091A8
:103808005F2B00915C2B10915D2B61D977DC0091C7
:10381800802BD4DF08959A938A9302E310E037DB74
:1038280056DB0EEF13E00E946B0A0F3F21F1F8946C
:1038380000E000939B2B00939A2B80E090E00AC055
:103848008C0100501E4F0E946B0A202F8C010E9491
:10385800B50A0196803002E0900794F32DE631E234
:1038680007EB15E20E94983C07EC0E94C40210E2A4
:1038780000E321DB0CC027E731E207EB15E20E94E9
:10388800983C07EC0E94C40210E500E214DB04E156
:103898000E94350308ED04BF01E000937900899187
:1038A800999108950E943F38F89400E30E94C90254
:1038B800E0E8F6E0008108600083009160060F6090
:1038C8000093600600914006006C00934006E0E615
:1038D800F6E0008100620083E0E4F6E00081026027
:1038E800008300916006006C0093600608E1009375
:1038F800110608E10093120608E10093130608E197
:103908000093300608E10093520608E1009353063D
:103918000E94EF010AEF11E00E946B0A0F3F11F4B9
:1039280001E001C000E0E8E0F6E0108111FD0CC004
:10393800E8E0F6E0108112FD07C0E8E2F6E0208139
:10394800217011E0212701C020E0022B002309F497
:10395800E2C021E831E207EB15E20E94983C00EC56
:103968000E94C402789402E30E943503F89400E0B0
:1039780000939B2BC3C021E001E010E00E94B50A30
:103988002FE802E010E00E94B50A20E005E010E010
:103998000E94B50A24EB06E010E00E94B50A20E078
:1039A80005E110E00E94B50A24EB06E110E00E9450
:1039B800B50A20E007E010E00E94B50A20EB08E015
:1039C80010E00E94B50A20E007E110E00E94B50A65
:1039D80020EB08E110E00E94B50A20E00EE010E0BC
:1039E8000E94B50A20E00FE010E00E94B50A20E02E
:1039F80000E110E00E94B50A20E001E110E00E9419
:103A0800B50A22E003E010E00E94B50A22E004E0D3
:103A180010E00E94B50A20E009EF11E00E94B50A03
:103A280027E00CE010E00E94B50A21E00DE010E06C
:103A38000E94B50A21E007EF11E00E94B50A21E0D3
:103A48000AE010E00E94B50A20E80BE010E00E94AE
:103A5800B50A20E00BEF11E00E94B50A28E10CEF4F
:103A680011E00E94B50A27E006EF11E00E94B50AAE
:103A780026E00DEF11E00E94B50A22E002E110E015
:103A88000E94B50A21E005EF11E00E94B50A21E085
:103A980003E110E00E94B50A20E008EF11E00E945F
:103AA800B50A22E00EEF11E00E94B50A24E004E115
:103AB80010E00E94B50A21E000E010E00E94B50A7B
:103AC80020E004EF11E00E94B50A20E003EF11E0C6
:103AD8000E94B50A20E00BE110E00E94B50A0091AF
:103AE8009A2B039500939A2B00919A2B033008F494
:103AF80042CF00919B2B039500939B2B00919B2B0E
:103B0800043020F400E000939A2BEECF20E00AEF77
:103B180011E00E94B50A0AEF11E00E946B0A0093B7
:103B28009B2B5ADE03E20093010807E0009300088C
:103B380006E910E0009326081093270880917C2B53
:103B480090E0019680932A0890932B0800917C2B93
:103B5800002331F400E010E00093260810932708B2
:103B680001E0009300090091852A1091862A0093AC
:103B780026091093270903E0009306090091A20083
:103B880007600093A20007E00093400804ED11E0ED
:103B9800009366081093670801E0009346080E94A6
:103BA8001B0300E10093220320915E2B30915F2BD1
:103BB80000915C2B10915D2B0E946B150E94F20204
:103BC80002E0009322020E9414030E940D030E9447
:103BD800F2020091802BF2DD91DA02E00E943503B7
:103BE80019DA0093942B1093952B03E20093410963
:103BF800009164060F730093640623E931E207EB32
:103C080015E20E94983C00EC0E94C40205E510E011
:103C18001A930A9324EA31E207EB15E20E94983CD2
:103C2800229600E80E94C40200ED17E00E942B17BC
:103C380000EA1FE00E942B1700E41FE10E942B17E7
:103C480008EE1DEF0E94561300ED17E00E942B1797
:103C580000E0009340090091A32A102F04E0109F70
:103C6800002D0E94350300E0009340090091B7251C
:103C78000B3409F0BACF0091B825003509F0B5CF5B
:103C88000091B9250F3409F0B0CF0091782B0023AB
:103C980031F0009164060F730093640605C000912B
:103CA8006406006C009364060091BA25043509F097
:103CB8009CCF0091A32A102F03E0109F002D0E9493
:103CC800350378940CE00E94240202E00E94350338
:103CD8003EDDE8E0F6E0008101FD24C0E8E0F6E022
:103CE800008102FD1FC00FEF00936E2B01E00093CF
:103CF8006D2B01E000936F2B01E00E94240210E578
:103D080000E30E945F1727EB31E207EB15E20E9400
:103D1800983C00E80E94C402E8E0F6E0008102FF57
:103D2800FBCF81C1E8E0F6E0008102FD21C00FEF82
:103D380000936E2B06E000936D2B02E000936F2B2F
:103D480001E00E94240210E500E30E945F1728ECBE
:103D580031E207EB15E20E94983C00E80E94C40299
:103D6800E8E0F6E0008102FFFBCF0E9467135BC129
:103D780000E000936F2B00E61AEE0E9456130ED94E
:103D88002801A091A32A6CC04091852A5091862AC7
:103D98004F5F5F4F652F660F660B762F00E01CE6BE
:103DA8002CED32E00E94AD3543E00E948235C80117
:103DB8005A924A9248EE53E08C010E9446351A9373
:103DC8000A9348EB5BE08C010E9446351A930A93EC
:103DD80023E032E207EB15E20E94983C269600E8C1
:103DE8000E94C4020091992A10919A2A1A930A9360
:103DF80026E132E207EB15E20E94983C229600EC9D
:103E08000E94C4020091832B10E0000F111FF801DB
:103E1800EF5DFC4F059114911A930A930091842B3E
:103E280010E01A930A930091802B10E0F801ED5EE0
:103E3800FC4F049110E01A930A9322E232E207EB56
:103E480015E20E94983C269609EC0E94C4020FECE9
:103E58000E9424020AE20E94680204E00E943503DC
:103E68000A2FA02FAA95002309F05CC001E00E9448
:103E7800240200E21EE40E94561305E0401600E00A
:103E880050060CF08FC02CE232E207EB15E20E94DC
:103E9800983C00E80E94C40200ED10E00E944B1715
:103EA80000EB10E00E944B1700ED10E00E944B174A
:103EB80004E10E943503B7C081E090E00091802BB7
:103EC80010E0F801ED5EFC4F049110E01A930A939C
:103ED8000091582B1091592B20915A2B30915B2B24
:103EE800021B130B1A930A930091542B1091552B14
:103EF8002091562B3091572B021B130B1A930A93C0
:103F08009A938A93B0E0BA93AA932CEE31E207EB26
:103F180015E20E94983C2A9600EC0E94C40207E031
:103F28000E943503E8E2F6E0008100FD2DCF08E0AD
:103F38000E9435036090992A70909A2A00917F2BED
:103F480010E01A930A935A924A927A926A9229ED49
:103F580031E207EB15E20E94983C269600E80E94A1
:103F6800C40200918A2B10918B2B013020E8120794
:103F780061F000E020918A2B30918B2B213010E0EA
:103F8800310719F00060002311F0A0E001C0A1E0A2
:103F980000915E2B10915F2B012B09F08DCF80E0F3
:103FA80090E08CCF0091992A10919A2A093522E045
:103FB8001207C8F10091992A10919A2A1A930A9324
:103FC8002AE332E207EB15E20E94983C229603E8C6
:103FD8000E94C40224E432E207EB15E20E94983CF6
:103FE80000EC0E94C40200ED10E00E944B1700EBA9
:103FF80010E00E944B1700ED10E00E944B17A1E063
:1040080010C008EE1DEF0E945613E8E0F6E00081AC
:1040180002FD06C00E94FA1510E200E30E945F1735
:10402800A395A23370F301E00093652B00E00093A1
:104038007A2B07E00093722B0093712B00E010E0BD
:1040480020E030E0EFE1FBE2008311832283338339
:10405800EBE0FBE2008311832283338300938B2AF6
:1040680010938C2A0093892A10938A2A212F220FD1
:10407800220B322FE3ECFAE200831183228333838D
:1040880001E010E000938C2B10938D2B03E00E942D
:10409800350300E310E00E944B1702E00E9435034D
:1040A80000E310E00E944B1700E010E00093A52AFF
:1040B8001093A62A01E00093702B20C0009164069B
:1040C800006C0093640600E20093532B01E0C00EDD
:1040D80000E0D01E8601680101342FE1120774F058
:1040E800CC24DD2434DB0091992A10919A2A0835D2
:1040F80022E0120718F401E00093652B00916E2B63
:10410800002309F084C30091702B013009F04DC2DF
:10411800E7EDFAE20081118122813381EFEFFAE2C3
:104128000083118322833383EBEDFAE2008111814E
:1041380022813381E3E1FBE200831183228333830D
:10414800E7EEFAE2008111810093832A1093842A12
:10415800E3EBFAE20081118122813381EBEFFAE28D
:104168000083118322833383E7EBFAE20081118114
:1041780022813381EFE0FBE20083118322833383C2
:10418800E3ECFAE2008111810093812A1093822ADC
:104198000091752B0D5F10917D2B011B0093772BE0
:1041A8000091772B10E02091812A3091822A021702
:1041B80013070CF0B9C10091772B10E02091832AE6
:1041C8003091842A021713070CF0AEC100916D2BB1
:1041D800002309F0A9C100E00093712B0091722B14
:1041E80003950093722B003118F001E00093652BC2
:1041F800E3E0FBE20081118122813381EBEFFAE2F7
:104208004081518162817381401B510B620B730B9A
:104218004083518362837383E7E1FBE2008111816C
:1042280022813381EFE0FBE2408151816281738119
:10423800401B510B620B730B408351836283738362
:10424800EBEFFAE20081118122813381EBEFFAE290
:1042580040815181628173810E945A35C801D90118
:10426800EFE0FBE20081118122813381EFE0FBE284
:1042780040815181628173810E945A35A801B90138
:104288008C019D01040F151F261F371F0E940F3632
:104298000E94B33C0E941C36159507951595079505
:1042A8000093902B1093912B1091912B11234AF48A
:1042B80022E104EF1EE70E94FF1600E21EE40E94BE
:1042C8005613E7E0FBE20081118122813381EFEF91
:1042D800FAE24081518162817381401B510B620B6C
:1042E800730B4083518362837383EBE1FBE20081AC
:1042F800118122813381E3E1FBE2408151816281B6
:104308007381401B510B620B730B40835183628393
:104318007383EFEFFAE20081118122813381EFEF9D
:10432800FAE240815181628173810E945A35C80145
:10433800D901E3E1FBE20081118122813381E3E1CC
:10434800FBE240815181628173810E945A35A80144
:10435800B9018C019D01040F151F261F371F0E94EC
:104368000F360E94B33C0E941C361595079515958B
:1043780007950093922B1093932B1091932B112355
:104388004AF422E104EF1EE70E94FF1600E21EE451
:104398000E945613EFE0FBE20081118122813381F4
:1043A8000E940F36A801B901CA01DB01EBEFFAE25E
:1043B80000811181228133810E940F36AC01BD0139
:1043C8000E9483170093872A1093882AE3E1FBE26F
:1043D80000811181228133810E940F36A801B90121
:1043E800CA01DB01EFEFFAE20081118122813381FA
:1043F8000E940F36AC01BD010E9483170093932AD7
:104408001093942A0091812A1091822A2091832A5C
:104418003091842A020F131F212F220F220B322FD3
:104428000E940F360E9465380E941C360093692B43
:1044380000916A2B002319F408E00093692B00917E
:104448006A2B023071F40091692B1091692B019F3E
:1044580080010D5F1F4F44E050E00E9446350093F5
:10446800692B0091812A1091822AE016F10624F521
:104478000091872A1091882A00938D2A10938E2AFA
:104488000091932A1091942A0093952A1093962AC2
:104498000091902B1091912B00938C2B10938D2BC6
:1044A8000091922B1091932B00938E2B10938F2BAE
:1044B800E090812AF090822A00918D2A10918E2A0C
:1044C80000938B2A10938C2A0093872A1093882AAA
:1044D8000091952A1091962A00938F2A1093902A7A
:1044E8000093932A1093942A0091862B1091722B93
:1044F800011738F40091932A1091942A0E94791A8E
:1045080086C100E010E000938F2A1093902A009350
:10451800932A1093942A00938B2A10938C2A009341
:10452800872A1093882A73C100E010E000936A0973
:1045380010936B09EBEFFAE200811181228133813C
:10454800E3E0FBE20083118322833383EFE0FBE2A5
:104558000081118122813381E7E1FBE2008311832D
:1045680022833383EFEFFAE20081118122813381C4
:10457800E7E0FBE20083118322833383E3E1FBE27C
:104588000081118122813381EBE1FBE200831183F9
:1045980022833383EE24FF240091712B039500932B
:1045A800712B00E00093722B32C1E7EDFAE2008133
:1045B800118122813381EBEFFAE200831183228398
:1045C8003383EBEDFAE20081118122813381EFE040
:1045D800FBE2008311832283338342E050E060E0F2
:1045E80070E0E3ECFAE200811181228133810E94BC
:1045F800AD350093812A1093822A42E050E060E0B2
:1046080070E0E7EEFAE200811181228133810E9495
:10461800AD350093832A1093842AEBEFFAE20081E8
:10462800118122813381EBEFFAE24081518162816D
:1046380073810E945A35C801D901EFE0FBE200817D
:10464800118122813381EFE0FBE240815181628157
:1046580073810E945A35A801B9018C019D01040F8C
:10466800151F261F371F0E940F360E94B33C0E9459
:104678001C3643E00E9428350093902B1093912B11
:104688000091752B10E02091812A3091822A02171F
:1046980013070CF0B1C00091752B10E02091832A0C
:1046A8003091842A021713070CF0A6C000916D2BD5
:1046B800002309F0A1C00091722B03950093722B7F
:1046C80000E00093712BEFE0FBE200811181228171
:1046D80033810E940F36A801B901CA01DB01EBEF53
:1046E800FAE200811181228133810E940F36AC01E8
:1046F800BD010E9483170093872A1093882A10917E
:10470800912B11234AF422E100E01DE70E94FF16D5
:1047180000E41CE90E9456130091812A1091822A14
:104728002091832A3091842A020F131F42E050E01F
:104738000E944635212F220F220B322F0E940F365E
:104748000E9465380E941C360093692B0091692BE2
:10475800083018F008E00093692B0091722B0430A0
:10476800C8F02091692BA22F80E49FE10091812A53
:104778001091822A2091832A3091842A020F131FD4
:1047880042E050E00E944635801B910B8C012A2F95
:104798000E94FF160091902B1091912B00938C2B67
:1047A80010938D2BE0918C2BF0918D2B3397ECF09F
:1047B800EFE0FBE200811181228133810E940F36F4
:1047C800A801B901CA01DB01EBEFFAE2008111810E
:1047D800228133810E940F36AC01BD010E948317EC
:1047E80000938B2A10938C2A12C000E010E00093EB
:1047F8008B2A10938C2A0BC000E00093400900E03C
:104808000093722B0091712B03950093712B0091EB
:10481800712B0C3D41F010E00091722B0C3D19F00A
:1048280010601123F9F000E010E000938C2B109336
:104838008D2B00938B2A10938C2A0093892A10932E
:104848008A2A00E010E000938E2B10938F2B0093A0
:104858008F2A1093902A0093912A1093922A01E0AC
:104868000093652B00916D2BE8E3F3E00C94FA3785
:1048780080918B2A90918C2A40908F2A5090902A70
:10488800E0918C2BF0918D2B33977CF0E0918E2B5F
:10489800F0918F2B33974CF08093892A90938A2A32
:1048A8004092912A5092922A08C08091892A909128
:1048B8008A2A4090912A5090922A0091822B0230A5
:1048C80009F07CC0840D951D8C0142E050E00E94E7
:1048D80046350E94BC1904E610E00E945613009168
:1048E8008C2B10918D2B212F220F220B322F0E94FF
:1048F8000F360E9465380E941C36C8010091712B42
:10490800053048F025E532E207EB15E20E94983CB5
:1049180007EC0E94C4021091912B112332F403E298
:10492800602E772489E090E00BC00091702B002363
:1049380021F40EE3602E772403C006E0602E77246E
:10494800A0E008C00A2F08530E942402062D0E94E6
:104958006802A395B0E0A817B907A4F30E943D1810
:1049680038014AE050E083010E9446355A934A9341
:104978004AE050E083010E9446351A930A93009159
:10498800532B10E01A930A9300917D2B10E01A9391
:104998000A930091752B10E01A930A930091762BD5
:1049A80010E01A930A932FE532E207EB15E20E9412
:1049B800983C2C9607E80E94C40292C5992352F0AD
:1049C8009A938A932FE632E207EB15E20E94983C0D
:1049D80022960EC04FEF5FEF8C010E9414351A9398
:1049E8000A9329E732E207EB15E20E94983C2296E7
:1049F80000E80E94C40200918C2B10918D2B212F6E
:104A0800220F220B322F0E940F360E9465380E9417
:104A18001C36C80199231AF483E290E006C0883056
:104A280000E0900711F48FEF90E004E80E94240260
:104A3800082F0E9468020091702B0130E9F555207B
:104A480052F05A924A9222E832E207EB15E20E94AB
:104A5800983C22960EC04FEF5FEF82010E941435FA
:104A68001A930A9329E732E207EB15E20E94983C71
:104A7800229600EC0E94C40200918E2B10918F2B7D
:104A8800212F220F220B322F0E940F360E946538E9
:104A98000E941C36C80199231AF483E290E006C0EC
:104AA800883000E0900711F48FEF90E004EC0E944A
:104AB8002402082F0E9468020091702B013009F02F
:104AC8007EC00091712B073090F02BE832E207EBA3
:104AD80015E20E94983C06E80E94C4022BE832E2E4
:104AE80007EB15E20E94983C06EC0E94C402109164
:104AF800882A112312F14AE050E00091872A109188
:104B0800882A0E9446350093972A1093982A009184
:104B1800972A0A570E94240200918C2B10918D2B02
:104B2800212F220F220B322F0E940F360E94653848
:104B38000E941C360E9468020DC01091882A112319
:104B48004AF426E932E207EB15E20E94983C06E8AF
:104B58000E94C4021091942A112312F14AE050E0F5
:104B68000091932A1091942A0E9446350093972A1F
:104B78001093982A0091972A0A530E9424020091C0
:104B88008E2B10918F2B212F220F220B322F0E9458
:104B98000F360E9465380E941C360E94680259C070
:104BA8001091942A11230AF054C026E932E207EB47
:104BB80015E20E94983C06EC0E94C4024AC043E0F9
:104BC8000091902B1091912B0E942835C801833CAD
:104BD80001E0900734F400E099231AF00060002304
:104BE80011F082EC91E02AE932E207EB15E20E942B
:104BF800983C00EC0E94C402A0E00FC00A2F0753A3
:104C08000E9424020EE30E94680206EC0A1B0E941E
:104C180024020CE30E946802A3950A2F10E020E00A
:104C280030E00E941A36280139018C01212F220F09
:104C3800220B322F0E940F360E946538A801B90155
:104C4800820193010E94D137C8F200ED17E00E945B
:104C580056130091A52A1091A62A0C3221E01207BA
:104C680078F50E943D1838014AE050E083010E941F
:104C780046355A934A934AE050E083010E944635EC
:104C88001A930A930091532B10E01A930A930091F8
:104C98007D2B10E01A930A930091752B10E01A935C
:104CA8000A930091762B10E01A930A932BEA32E2CA
:104CB80007EB15E20E94983C2C9607E80E94C40274
:104CC8000FC480919B2B90E001969A938A932BEBCB
:104CD80032E207EB15E20E94983C229600E80E9417
:104CE800C40207E80E942402A0E009C00A2F10E0CD
:104CF80000541E4F0E946B0A0E946802A395A930B7
:104D0800A8F300E21EE40E945613E8E2F6E00081F0
:104D180000FD6CC008E210E00E944B170DE00E94F5
:104D28002402A0E407E000937A2B0FC000917A2BAD
:104D3800039500937A2B003118F00FE000937A2B3B
:104D4800A0E408E210E00E944B1700917A2B00586B
:104D58000E94240206E00E943503E8E0F6E00081A4
:104D680002FFE4CFE8E0F6E0008101FD10C0009109
:104D78007A2B0A9500937A2B073018F407E00093F2
:104D88007A2BA0E408E210E00E944B17DECFE8E29D
:104D9800F6E0008100FD1EC0A3950A2FA02F0B3559
:104DA80008F0A0E3AA3309F4A0E20A2F0E946802DF
:104DB80000917A2B00580E94240202E310E00E941E
:104DC8004B172A2F00917A2B10E007541E4F0E9490
:104DD800B50ABBCFE8E0F6E0008103FDB6CF08E2F4
:104DE80010E00E944B170CE00E9424020E946713F7
:104DF80024EC32E207EB15E20E94983C00EC0E949A
:104E0800C402A0E010C00A2F09530E9424020A2FEE
:104E18000E946802A83031F40EEC0E9424020FEFC1
:104E28000E946802A39580919B2B90E00196B0E0C8
:104E38008A179B0744F754C30E943D18C8014AE0EB
:104E480050E08C010E9446355A934A934AE050E05C
:104E58008C010E9446351A930A930091732B10E037
:104E6800F801E25FFC4F04914AE00E94F63450E0FA
:104E78005A934A930091732B10E0F801E25FFC4FBC
:104E880004914AE00E94F63410E01A930A9325ED43
:104E980032E207EB15E20E94983C289600E80E944F
:104EA800C4020091792B10E01A930A932BEE32E298
:104EB80007EB15E20E94983C229600EC0E94C4027F
:104EC80002E00E9435030CC300917C2B10E01A937A
:104ED8000A932CEF32E207EB15E20E94983C2296E7
:104EE80000E80E94C4022EE033E207EB15E20E94BC
:104EF800983C00EC0E94C402A0E010C00A2F0A539C
:104F08000E9424020A2F0E946802A83031F40EEC95
:104F18000E9424020FEF0E946802A39500917C2B47
:104F28000A1760F702E00E943503DAC20E94D2171E
:104F3800C8014091852A5091862A4F5F5F4F652F9F
:104F4800660F660B762F00E01CE62CED32E00E941F
:104F5800AD3543E00E94823528019A938A9320E276
:104F680033E207EB15E20E94983C229600E80E9483
:104F7800C4025A924A9243E050E082010E944635A8
:104F88001A930A9323E333E207EB15E20E94983C55
:104F9800249600EC0E94C40200E41CE90E94561307
:104FA8009FC28091632B90E001969A938A9320E4A4
:104FB80033E207EB15E20E94983C229600E80E9433
:104FC800C40222E533E207EB15E20E94983C00ECAC
:104FD8000E94C4020FED10E01A930A930091582B17
:104FE8001091592B1A930A930FED10E01A930A9314
:104FF8000091542B1091552B1A930A932AE533E20A
:1050080007EB15E20E94983C289607EC0E94C40220
:1050180000E41CE90E94561363C20E94D2171A9337
:105028000A9327E633E207EB15E20E94983C2296A2
:1050380000E80E94C4022FE633E207EB15E20E9463
:10504800983C07E80E94C40229E733E207EB15E21F
:105058000E94983C00EC0E94C402A0E010C00A2FF5
:105068000A530E9424020A2F0E946802A83031F4D1
:105078000EEC0E9424020FEF0E946802A395009193
:10508800812B0A1760F702E00E94350329C20091BC
:10509800842B10E01A930A930091802B10E0F801FA
:1050A800ED5EFC4F049110E01A930A932AE833E26C
:1050B80007EB15E20E94983C249600E80E94C4027F
:1050C80023E933E207EB15E20E94983C06E80E94C8
:1050D800C4022EE933E207EB15E20E94983C00EC8B
:1050E8000E94C402A0E010C00A2F0A530E942402A2
:1050F8000A2F0E946802A83031F40EEC0E942402A4
:105108000FEF0E946802A3950091802B0A1760F7A1
:1051180002E00E943503E4C10091992A10919A2A6D
:105128001A930A932FEA33E207EB15E20E94983CA0
:10513800229600E80E94C40200915E2B10915F2B1A
:105148001A930A932AEB33E207EB15E20E94983C84
:10515800229609E80E94C4020FED10E01A930A9300
:1051680000915C2B10915D2B1A930A9325EC33E286
:1051780007EB15E20E94983C249600EC0E94C402BA
:10518800AFC10091742B10E01A930A932AED33E211
:1051980007EB15E20E94983C229600E80E94C402A0
:1051A80023E933E207EB15E20E94983C06E80E94E7
:1051B800C40222EE33E207EB15E20E94983C00ECB1
:1051C8000E94C402A0E010C00A2F0A530E942402C1
:1051D8000A2F0E946802A83031F40EEC0E942402C3
:1051E8000FEF0E946802A3950091742B0A1760F7CD
:1051F80002E00E94350374C123EF33E207EB15E2A6
:105208000E94983C00E80E94C4022AE034E207EBBE
:1052180015E20E94983C00EC0E94C40261C1009112
:105228006A2B10E0000F111FF801E35DFC4F059198
:1052380014911A930A932BE134E207EB15E20E94CA
:10524800983C229600E80E94C40223E933E207EB67
:1052580015E20E94983C06E80E94C40222E234E269
:1052680007EB15E20E94983C00EC0E94C402A0E003
:1052780010C00A2F0A530E9424020A2F0E946802B3
:10528800A83031F40EEC0E9424020FEF0E9468024D
:10529800A39500917B2B0A1760F700E61AEE0E948F
:1052A80056131EC100917E2B033019F48AE090E05A
:1052B80005C080917E2B90E0880F991F00917E2B6E
:1052C800043039F423E334E207EB15E20E94983CFA
:1052D80009C09A938A932AE334E207EB15E20E9405
:1052E800983C229600E80E94C40223E933E207EBC7
:1052F80015E20E94983C06E80E94C40222E434E2C7
:1053080007EB15E20E94983C00EC0E94C402A0E062
:1053180010C00A2F0A530E9424020A2F0E94680212
:10532800A83031F40EEC0E9424020FEF0E946802AC
:10533800A39500917E2B0A1760F702E00E943503BF
:1053480000917E2B053081F48EE591E009C08093B1
:1053580026099093270908EB1BE00E945613049630
:10536800883E03E090079CF3BBC00091852B10E0BA
:105378001A930A930091822B10E0000F111FF80175
:10538800EF5CFC4F059114911A930A9323E534E2DC
:1053980007EB15E20E94983C249600E80E94C4029C
:1053A80023E634E207EB15E20E94983C00EC0E94E9
:1053B800C402A0E010C00A2F0A530E9424020A2F38
:1053C8000E946802A83031F40EEC0E9424020FEF0C
:1053D8000E946802A3950091852B0A1760F702E0E6
:1053E8000E9435037DC00091862B10E01A930A9322
:1053F8000091832B10E0000F111FF801EF5DFC4FA7
:10540800059114911A930A9324E734E207EB15E205
:105418000E94983C249600E80E94C40223E834E2E3
:1054280007EB15E20E94983C00EC0E94C402A0E041
:1054380010C00A2F07530E9424020A2F0E946802F4
:10544800A83031F40EEC0E9424020FEF0E9468028B
:10545800A3950091862B0A1760F702E00E94350396
:1054680001E00093672B3CC00091672B0023C1F13A
:1054780024E934E207EB15E20E94983C00E80E9418
:10548800C402A0E004C000E20E946802A395A03113
:1054980090F40A2F00540E9424024A2F00918A2B6C
:1054A80010918B2B0E9428350170002361F303E2D1
:1054B8000E946802EBCF05EC0E9424020FE20E94D2
:1054C800680200917A2B00540E9424020EE00E9488
:1054D800240200E00093672B08EE1DEF0E9456138C
:1054E800B0E0E8E0F6E0008103FDCEC000E0009304
:1054F800400901E00093652B00E010E00093A52A25
:105508001093A62A00916B2B0130B1F406E210E04B
:105518000E944B17E8E0F6E0008103FFFBCF01E0B3
:105528000093652B04EB0093722B0093712B00E022
:1055380000936B2B0C944734E8E0F6E0008103FD00
:1055480054C008EE1DEF0E945613B3950B2FB02FD1
:105558002091A32A3091A42A10E02017310760F780
:1055680000916E2B009500936E2B01E000936B2B3E
:105578000091822B023019F40E948B1302C00E9402
:10558800671301E00E94240200916E2B002381F42E
:1055980000E000936D2B4091812B50E00FEF10E05D
:1055A8000E9414350E94E91402E00E94350309C0E4
:1055B8000BE000936D2B08EE1DEF0E9456130E941E
:1055C800671301E00093672B00E000936F2B00E066
:1055D8000093702B0AE510E00E944B1701E000933E
:1055E800652B01E00093702B3CC200916E2B0023C9
:1055F80069F40091702B00950093702B0E94511B49
:1056080004EB0093722B0093712B38C00CE00E94BE
:10561800240200916F2B013059F400916D2B0395F2
:1056280000936D2B0B30E8F001E000936D2B19C04F
:1056380000916F2B023059F400916D2B0395009364
:105648006D2B0B3070F008E000936D2B0AC00091B1
:105658006D2B039500936D2B003118F001E000933A
:105668006D2B00916D2B083049F44091812B50E04F
:105678000FEF10E00E9414350E94E91408E210E0D0
:105688000E944B170C944434E8E2F6E0008100FDD8
:10569800CCC400E00093400900E010E00093A52A84
:1056A8001093A62A08EC0093712B00916D2B0050E3
:1056B800F9F0025009F4DFC1025009F4F7C10A9564
:1056C80009F43EC2025009F4B7C30A9509F4CCC3E1
:1056D800025009F4D1C30A9509F411C4025009F41F
:1056E80027C40A9509F43CC40A9509F457C495C41B
:1056F80001E00E94240200E21EE40E945613E8E240
:10570800F6E0008100FD0FC000E61AEE0E94561375
:10571800B3950B2FB02F2091A32A3091A42A10E023
:105728002017310760F7B3950B2FB02F2091A32ACC
:105738003091A42A10E02017310708F063C100E374
:1057480010E00E944B17EFEBFAE2008111812281F1
:1057580033810E940F36A801B901CA01DB01EBEBC6
:10576800FAE200811181228133810E940F36AC0157
:10577800BD010E9483170093872A1093882AEBEBB8
:10578800FAE20081118122813381EBE0FBE20083A0
:10579800118322833383EFEBFAE2008111812281A6
:1057A8003381EFE1FBE20083118322833383E3EE4D
:1057B800FAE200811181228133810E940F36A8010B
:1057C800B901CA01DB01EFEDFAE200811181228102
:1057D80033810E940F36AC01BD010E9483170093EC
:1057E800932A1093942AEFEDFAE200811181228125
:1057F8003381E7E0FBE20083118322833383E3EE06
:10580800FAE20081118122813381EBE1FBE200831E
:105818001183228333830091922B1091932B212F94
:10582800220F220B322F0E940F360E946538C801C2
:10583800D9010091902B1091912B212F220F220B2F
:10584800322F0E940F360E946538280139010091D5
:10585800932A1091942A1A930A930091872A1091F7
:10586800882A1A930A9340E050E060E070E48C01C3
:105878009D010E94CF360E941C361A930A9340E07D
:1058880050E060E070E4820193010E94CF360E94EC
:105898001C361A930A9325EA34E207EB15E20E94B4
:1058A800983C289600E80E94C4020091872A10912B
:1058B800882A053C2FEF120704F500E02091872A7B
:1058C8003091882A263A1FEF3107BCF010E020916A
:1058D800932A3091942A253C4FEF340774F420E042
:1058E8004091932A5091942A463A3FEF53072CF05F
:1058F800012B022B00600023D9F02DEB34E207EBDB
:1059080015E20E94983C00EC0E94C40200EA10E0F4
:105918000E944B1700EB10E00E944B17E8E2F6E0FC
:10592800008100FD8FC0E8E0F6E0008103FDF6CFBE
:105938002EEC34E207EB15E20E94983C00EC0E9442
:10594800C40200E210E00E944B170091542B109102
:10595800552B2091872A3091882A021B130B0A5550
:1059680010400093562B1093572B0091582B1091F1
:10597800592B2091932A3091942A021B130B0A5514
:10598800104000935A2B10935B2B1091572B112327
:1059980042F4E6E5FBE20081118108591E4F0083BD
:1059A800118310915B2B112342F4EAE5FBE200819D
:1059B800118108591E4F008311830E948218E8E262
:1059C800F6E0008100FFFBCF3091572B232F07E033
:1059D80010E00E94B50A2091562B08E010E00E94C2
:1059E800B50A30915B2B232F07E110E00E94B50A1E
:1059F80020915A2B08E110E00E94B50A06E00E94A7
:105A0800350320C001E00093652B0091992A10917D
:105A18009A2A1A930A932FED34E207EB15E20E94B3
:105A2800983C229600E80E94C40200E310E00E941D
:105A38004B170091722B002311F401E001C000E024
:105A48000093712B08E00E94350301E00093652B59
:105A580021EF34E207EB15E20E94983C00EC0E942B
:105A6800C40222E035E207EB15E20E94983C00E808
:105A78000E94C40205C70091732B03950093732BF2
:105A8800053018F000E00093732B2091732B0EEF74
:105A980011E00E94B50A0091A32A1091A42A0E943D
:105AA800561302E310E00E944B17EAC6A0E0B0E0EC
:105AB8000E946B1786E791E012C0809326099093A5
:105AC800270904E00E9435030E94D217A017B107E6
:105AD8002CF4D8018093852A9093862A04968939D4
:105AE80002E0900754F30091852A1091862A0093CA
:105AF8002609109327090E94511B10E400E50E9413
:105B08005F173091862A232F01E010E00E94B50A22
:105B18002091852A02E010E00E94B50AB1C62AE267
:105B280035E207EB15E20E94983C00E80E94C402A7
:105B380000E810E00E944B1700E810E00E944B17A5
:105B4800E8E2F6E0008100FD64C100E61AEE0E947A
:105B58005613B3950B2FB02F2091A32A3091A42A66
:105B680010E02017310760F701E00093682B28E068
:105B780035E207EB15E20E94983C00E80E94C40257
:105B880000E310E00E944B1701E00093652B0091A1
:105B9800A32A102F02E0109F002D0E94350329E14F
:105BA80035E207EB15E20E94983C00E80E94C40227
:105BB80000E310E00E944B170091A32A0E943503CE
:105BC80000E010E02801C801A0E038C0EFEBFAE2DD
:105BD80000811181228133810E940F36A801B90109
:105BE8004A015B01EBEBFAE20081118122813381EA
:105BF8000E940F36A401B5010E947817800F911FEB
:105C0800E3EEFAE200811181228133810E940F368E
:105C1800A801B9014A015B01EFEDFAE200811181A7
:105C2800228133810E940F36A401B5010E947817A2
:105C3800400E511E06E00E943503A395AA3030F2AB
:105C48004AE050E08C010E944635C8014AE050E025
:105C580082010E9446352801E091542BF091552B82
:105C6800EA55F040E81BF90BE093542BF093552BC1
:105C78000091542B1091552B093621E0120744F05E
:105C8800E4E5FBE20081118108561140008311838D
:105C98001091552B112342F4E4E5FBE200811181B8
:105CA80008591E4F008311838091582B9091592BCE
:105CB8008A559040841995098093582B9093592BB5
:105CC8000091582B1091592B093621E0120744F006
:105CD800E8E5FBE200811181085611400083118339
:105CE8001091592B112342F4E8E5FBE20081118160
:105CF80008591E4F008311830E9453180091A32A4C
:105D08000E943503EFEBFAE2008111812281338191
:105D18000E940F36A801B9014A015B01EBEBFAE2D8
:105D280000811181228133810E940F36A401B501BF
:105D38000E947817C801E3EEFAE2008111812281FE
:105D480033810E940F36A801B9014A015B01EFEDCA
:105D5800FAE200811181228133810E940F36A40169
:105D6800B5010E947817400E511E8C3A0FEF90072C
:105D78000CF0D5CE0CEA40160FEF50060CF0CFCE43
:105D88002BE335E207EB15E20E94983C00E80E94FD
:105D9800C40205E210E00E944B1705E00E9435039B
:105DA80005E210E00E944B173091552B232F05E098
:105DB80010E00E94B50A2091542B06E010E00E94E2
:105DC800B50A3091572B232F07E010E00E94B50A3F
:105DD8002091562B08E010E00E94B50A3091592B0B
:105DE800232F05E110E00E94B50A2091582B06E107
:105DF80010E00E94B50A30915B2B232F07E110E0D9
:105E08000E94B50A20915A2B08E110E00E94B50AB9
:105E180097CE0091682B002371F40091632B0395B2
:105E28000093632B023018F000E00093632B00E529
:105E380010E00E944B1724C50091842B0395009312
:105E4800842B033018F001E00093842B2091842BDD
:105E580000E010E00E94B50A02E310E00E944B1730
:105E680004E00E9435030CC501E00093652B02E3B2
:105E780010E00E944B1704C5E8E2F6E0008100FD3F
:105E88003EC008EE1DEF0E945613B3952B2FB22F7C
:105E98000091A32A1091A42A000F111F30E00217C5
:105EA800130750F710E400E30E945F17F89400E02E
:105EB80000939B2B00939A2B80E090E00AC08C0102
:105EC8000E946B0A202F8C0100501E4F0E94B50AB9
:105ED8000196803002E0900794F32CE435E207EB5A
:105EE80015E20E94983C00EC0E94C402789410E2EB
:105EF80000E30E945F170AE00E943503B2CD0091CB
:105F08006A2B039500936A2B033018F000E0009386
:105F18006A2B20916A2B08EF11E00E94B50A02E370
:105F280010E00E94561302E310E00E944B17A8C429
:105F38000091822B03950093822B033018F001E027
:105F48000093822B2091822B05EF11E00E94B50A65
:105F580002E310E00E944B1704E00E94350390C44E
:105F68000091832B03950093832B043018F001E0F4
:105F78000093832B0091802B0E94E21B2091832B9E
:105F880003E110E00E94B50A0E94511B02E310E0F1
:105F98000E944B1706E00E94350372C481E090E02E
:105FA80040917A2B8C010E941C35C80140917A2BB4
:105FB80000918A2B10918B2B0E94283501700023A9
:105FC80079F080959095EAE8FBE200811181082339
:105FD80019230083118310E500E40E945F170CC0A9
:105FE800EAE8FBE200811181082B192B0083118359
:105FF80010E300E40E945F1701E00093672B2091F3
:106008008A2B0AE010E00E94B50A30918B2B232FCF
:106018000BE010E00E94B50A33C401E00093652B41
:1060280008E210E00E944B172BC4E8E0F6E000817C
:1060380002FD19C200E00093400900E010E000935F
:10604800A52A1093A62A00916D2BEEE5F3E00C9497
:10605800FA37E8E0F6E0008102FD25C000E61AEE16
:106068000E945613B3950B2FB02F2091A32A30917D
:10607800A42A10E02017310760F70091782B0095CB
:106088000093782B2091782B09EF11E00E94B50A34
:1060980001E00093682B00E510E00E944B1701E037
:1060A8000E943503F0C30091682B002381F400910E
:1060B800752B03950093752B0A3018F000E00093B8
:1060C800752B2091752B03E010E00E94B50AC3C11F
:1060D80000919B2B039500939B2B043018F003E051
:1060E80000939B2B0E94F01B20919B2B0AEF11E041
:1060F8000E94B50AB0C10091792B03950093792BC2
:106108000D3318F001E00093792B2091792B0CEFD7
:1061180011E00E94B50A00E41CE90E9456139BC1D5
:1061280000917C2B039500937C2B093018F008E034
:1061380000937C2B0BE910E00093260810932708A6
:1061480020917C2B0DEF11E00E94B50A80917C2BE9
:1061580090E0019680932A0890932B087CC1809147
:10616800852A9091862A01978093852A9093862A7A
:10617800863701E0900734F406E711E00093852A9A
:106188001093862A0091852A1091862A0093260961
:10619800109327090E94511B3091862A232F01E072
:1061A80010E00E94B50A2091852A02E010E00E94C2
:1061B800B50A51C10091632B002319F58091542B26
:1061C8009091552B01968093542B9093552B89369B
:1061D80001E0900734F000E010E00093542B109396
:1061E800552B0E9453183091552B232F05E010E0B2
:1061F8000E94B50A2091542B06E010E00E94B50ACF
:106208002AC18091582B9091592B01968093582B35
:106218009093592B893601E0900734F000E010E0A4
:106228000093582B1093592B0E9453183091592BD7
:10623800232F05E110E00E94B50A2091582B06E1B2
:1062480010E00E94B50A07C10091812B03950093C5
:10625800812B083018F007E00093812B4091812BA7
:1062680050E00FEF10E00E9414350E94E9142091CD
:10627800812B0CE010E00E94B50AEDC00091802B44
:1062880003950093802B053018F004E00093802BD1
:106298000091802B0E94E21B2091802B02E110E0EC
:1062A8000E94B50AD8C0E8E0F6E0008101FD1BC0F5
:1062B80000E010E000935E2B10935F2B00935C2BA3
:1062C80010935D2B04E610E00E944B1706E00E9435
:1062D800350320E00EE010E00E94B50A20E00FE050
:1062E80010E00E94B50A0091642B002309F5809103
:1062F8005E2B90915F2B019680935E2B90935F2B82
:10630800813008E0900734F000E018E000935E2B3D
:1063180010935F2B30915F2B232F00E110E00E9438
:10632800B50A20915E2B01E110E00E94B50A20C059
:1063380080915C2B90915D2B019680935C2B9093C0
:106348005D2B883601E0900734F000E010E0009300
:106358005C2B10935D2B30915D2B232F0EE010E00A
:106368000E94B50A20915C2B0FE010E00E94B50A4C
:1063780020915E2B30915F2B00915C2B10915D2B4F
:106388000E946B1502E00E94350365C00091742BD2
:1063980003950093742B093018F008E00093742BD0
:1063A8002091742B04E110E00E94B50A54C00E94A9
:1063B8000F1C51C000917B2B039500937B2B093058
:1063C80018F008E000937B2B20917B2B06EF11E05F
:1063D8000E94B50A40C000917E2B039500937E2B46
:1063E800053018F004E000937E2B20917E2B07EFF8
:1063F80011E00E94B50A2FC00091852B03950093E8
:10640800852B093018F008E00093852B2091852B07
:1064180003EF11E00E94B50A1EC00091862B039578
:106428000093862B063018F005E00093862B209108
:10643800862B0BE110E00E94B50A0DC000917A2B63
:10644800039500937A2B003118F000E000937A2B23
:1064580001E00093672B08E210E00E944B1701E06F
:106468000093652B0DC2E8E0F6E0008101FD08C24B
:1064780000E00093400900E010E00093A52A109383
:10648800A62A00916D2BE4E8F3E00C94FA37E8E0D3
:10649800F6E0008101FD2AC000E61AEE0E945613BC
:1064A800B3950B2FB02F2091A32A3091A42A10E086
:1064B8002017310760F700917D2B039500937D2B02
:1064C800043018F001E000937D2B20917D2B0DE026
:1064D80010E00E94B50A01E00093682B00E510E087
:1064E8000E944B1703E00E943503CDC10091682B31
:1064F800002381F40091762B03950093762B0A30C4
:1065080018F000E00093762B2091762B04E010E041
:106518000E94B50AAEC100919B2B0A9500939B2B54
:106528000F3F19F400E000939B2B0E94F01B209171
:106538009B2B0AEF11E00E94B50A9BC10091792BB1
:106548000A950093792B002319F40CE30093792B17
:106558002091792B0CEF11E00E94B50A00E41CE9A8
:106568000E94561386C100917C2B0A9500937C2BC0
:106578000F3F19F400E000937C2B20917C2B0DEF4A
:1065880011E00E94B50A80917C2B90E001968093DF
:106598002A0890932B086DC18091852A9091862AAC
:1065A80001968093852A9093862A8A3902E090077B
:1065B80034F009E912E00093852A1093862A0091A5
:1065C800852A1091862A00932609109327090E948C
:1065D800511B3091862A232F01E010E00E94B50A52
:1065E8002091852A02E010E00E94B50A42C100917C
:1065F800632B002309F58091542B9091552B01971B
:106608008093542B9093552B992332F408E611E08C
:106618000093542B1093552B0E9453183091552BEF
:10662800232F05E010E00E94B50A2091542B06E0C4
:1066380010E00E94B50A1DC18091582B9091592BEA
:1066480001978093582B9093592B992332F408E69D
:1066580011E00093582B1093592B0E945318309136
:10666800592B232F05E110E00E94B50A2091582BE1
:1066780006E110E00E94B50AFCC00091812B0A9542
:106688000093812B0F3F19F400E00093812B409178
:10669800812B50E00FEF10E00E9414350E94E9149E
:1066A8002091812B0CE010E00E94B50AE2C0009115
:1066B800802B0A950093802B013018F401E0009399
:1066C800802B0091802B0E94E21B2091802B02E1FD
:1066D80010E00E94B50ACDC0E8E0F6E0008102FDB6
:1066E80011C000E010E000935E2B10935F2B009325
:1066F8005C2B10935D2B04E610E00E944B1706E01C
:106708000E9435030091642B0023F9F480915E2BDD
:1067180090915F2B019780935E2B90935F2B992329
:1067280032F400E010E000935E2B10935F2B309161
:106738005F2B232F00E110E00E94B50A20915E2B09
:1067480001E110E00E94B50A1EC080915C2B909177
:106758005D2B019780935C2B90935D2B992332F4EA
:1067680007E611E000935C2B10935D2B30915D2BB5
:10677800232F0EE010E00E94B50A20915C2B0FE059
:1067880010E00E94B50A20915E2B30915F2B00919A
:106798005C2B10915D2B0E946B1502E00E94350363
:1067A80068C00091742B0A950093742B0F3F19F45D
:1067B80000E00093742B2091742B04E110E00E94F8
:1067C800B50A57C008ED04BF01E00093790051C035
:1067D80000917B2B0A9500937B2B0F3F19F400E067
:1067E80000937B2B20917B2B06EF11E00E94B50ACA
:1067F80040C000917E2B0A9500937E2B013018F43F
:1068080001E000937E2B20917E2B07EF11E00E9480
:10681800B50A2FC00091852B0A950093852B0F3F51
:1068280019F400E00093852B2091852B03EF11E0EC
:106838000E94B50A1EC00091862B0A950093862BEC
:106848000F3F19F400E00093862B2091862B0BE173
:1068580010E00E94B50A0DC000917A2B0A950093AA
:106868007A2B0F3F19F40FE000937A2B01E0009385
:10687800672B08E210E00E944B1701E00093652B9C
:1068880000E00093682B0091782B002311F40C94FE
:106898006220009164060F73009364060AE2009375
:1068A800532B0C946A2000008895FECF0E9447382D
:1068B800C801D9012A013B015CD057D071F482018B
:1068C800930153D051F401E2E2EAFBE200834183F1
:1068D8000FEF1FEF2FE73FE73DC044D0A201B30100
:1068E8000E946E36AC01BD0140D061F442D03AD06E
:1068F8000E94E9370BED1FE029EC10F43FE32AC0B2
:106908003FEB28C0A201B3012DD00E9448370801EF
:1069180019012FD0820193010E94D13723D0A0F40E
:106928001CD050F424D0A801B9010BED1FE029E4D4
:1069380030E40E94B2360EC01AD04BED5FE069E435
:1069480070EC0E946E3606C008D010F410D002C059
:106958000ED03058E8E00C9458380E94E93780018E
:10696800910108958C019D0108950C94C7370C94EA
:10697800493B40E050E060E070E008953F7741E037
:106988000C94E83B03E20DBF01E20EBFC0E0D1E288
:106998000E94E838002311F00E94CB3B0E94561C4D
:1069A8000E9457340C9457340D01DA0140E050E04E
:1069B80060E070E00E94C73739F400E010E04D93C2
:1069C8004C9320E030E00CC0B901660F771F7E576A
:1069D800572F550F550B7D935C932F7730783F6376
:1069E800D00108950024E8E0EA9532F0001F001C69
:1069F8000416D0F3041AF8CF001F402D009508950F
:106A0800FF27442312F4F1604195002312F4F09516
:106A180001950E94F634F0FD0195F1FD4195089528
:106A2800149F102D059F100D049F002D110D089522
:106A38004A951AF0000F111FFBCF08954A951AF0D6
:106A480016950795FBCF08954A951AF01595079561
:106A5800FBCF089500241124EFE0001F111F001C34
:106A6800111C0416150610F0041A150AEA95AAF75F
:106A7800001F111FA001009510950895519541958B
:106A880050400895FF27552312F4F160F7DF1123D2
:106A980012F4F09507D00E942E35F0FD03D0F1FDD9
:106AA800EDCF089511950195104008952224349F43
:106AB800302D259F300D169F300D079F300D249FD8
:106AC800202D310D159F200D311D069F200D311DE4
:106AD800149F102D210D321D059F100D211D321DF3
:106AE800049F002D110D221D321D08954A952AF08C
:106AF8003695279517950795F9CF08954A952AF061
:106B08003595279517950795F9CF089500241124F1
:106B18001001E0E2EA9592F0001F111F221F331FB7
:106B2800001C111C221C331C0416150626063706E9
:106B380088F3041A150A260A370AECCF001F111F1A
:106B4800221F331FA001B1010095109520953095A3
:106B58000895FF27772312F4F16015D0332312F438
:106B6800F09509D00E948A35F69508F404D0F69578
:106B780008F409C0089530952095109501951F4F88
:106B88002F4F3F4F089570956095509541955F4FF1
:106B98006F4F7F4F0895FF27112477FB660F771FEC
:106BA800089409F4771F679517F8EE27002437FB38
:106BB800220F331F089409F4331F279507F8089507
:106BC80027FD0EC0EE0F001F111F221F3A9532300D
:106BD800B8F7332319F427FD31E002C027FF30E06E
:106BE800E03821F400FF08940EF488940F4F1F4FEB
:106BF8002F4F3F4F323038F4332319F427FD31E05B
:106C080002C027FF30E03F3F29F0220F000C3795E4
:106C180027950895ACC0032E002012F40E94BF35BA
:106C2800E02F012F122F232F3EE9D1CF0024F8CFD8
:106C3800BCDF432F4F5748F04F3148F007FC91C055
:106C48003FE72FEF1FEF0FEF089533278CC0322F48
:106C5800212F102F0E2F4F5141950E947A3507FE94
:106C680008950C94BF35F901EE0FFF1F37FBFF3F66
:106C780031F0EF2BE12BE02B8894B8940895E02BAA
:106C8800E12B21F008949894B894089598948894E6
:106C980038940895FB01EE0FFF1F77FBFF3F31F09B
:106CA800EF2BE52BE42B8894B8940895E42BE52B7F
:106CB80069F3E8CFEFDF68F021F43723262F8A0144
:106CC8000895372FFBCFE6DF20F00BF008957327E8
:106CD800EAF751C0C8DFE8F3B3F361F3DBDFC8F3C9
:106CE80083F3A1F358DF401751076207730731F4A4
:106CF800011411F10024E89488942BC078F0332E05
:106D0800372F732D322E262F632D312E152F532D0D
:106D1800302E042F432D302C012C132C371739F02B
:106D2800669557954795F795E0407395F7CFE7FB3C
:106D3800EE0FE0E010246AF0EF0F041F151F261F66
:106D480060F4279517950795E79508F468943395A7
:106D58003ECFEF0B040B150B260B39CFE0E87E274F
:106D6800B9CF302D307822271127002708953FE723
:106D7800302920E8F9CF3FEF2FEFF6CF8BDFD8F39C
:106D8800D1F370783727089585DFA8F3A3F3F9CFF7
:106D98003078372793CF67DF70F383F3A9F37ADF6F
:106DA80050F3B3F3A9F3F7DE0124E8943F57E0402A
:106DB800370FEF1F12F0D9F603C03A3E90F26894ED
:106DC800E0E00A92AA933A93AA273324222433278D
:106DD800049FF001059FF00D712D731F149FF00D96
:106DE800711D221C069F700D211C331C159F700DF0
:106DF800211C331E249F700D211C331E169F200C4E
:106E0800311CAA1F259F200C311CA31F269F300C64
:106E1800A11D39915EF43395A695379427947795FB
:106E2800F795E79533953130BCF316C0AA2322F0C5
:106E3800332351F4339510C0339571F4A991099017
:106E480096CFA7FD09C03A95EE0FFF1F771F221CAA
:106E5800331CAA1F3230A8F7E894FE2B09F0689477
:106E68002A2F8101E72FA9910990BACE13DF10F0DC
:106E78000BF087CF80CF0EDFE9F3E0F3032E072670
:106E880070CF032E072673CFEEDEA0F37BF399F3C2
:106E980001DF80F39BF3A9F37EDE012427FD06C002
:106EA800000F111F221F3150E040F8CF67FD06C0C8
:106EB800440F551F661F7150F040F8CFE894371BF8
:106EC800EF0B3158EF4F2AF0EE23E9F63F3FD9F2A6
:106ED80003C03A3EA8F26894E0E0F0E0112413946D
:106EE80040175107620738F0315008F46894000FD2
:106EF800111F221FEE1F041B150B260BEF0B000F93
:106F0800111F221FEE1F0A9279E17A95AAF0041741
:106F180015072607EF0730F0041B150B260BEF0BA0
:106F2800089401C08894111C221C331C001C000FFB
:106F3800111F221FEE1FE9CFF0F9E894E22BE12B95
:106F4800E02B09F068940694379427941794E795F2
:106F580008F468947395B9F30990332311F0F0FF9E
:106F680009C0369427941794E79508F468943395E4
:106F78003130BCF3012D122D232D32CE8BCE9894B7
:106F88000895189408956FDED0F3C1F383DEB8F343
:106F9800041715072607370708957CDEA0F063DE7F
:106FA80090F029F0E32FE7273AF47317089572DE7B
:106FB80051F04EF00894089504171507260737076F
:106FC80019F016F4B8F78894089564DEE0F34BDE00
:106FD800D0F3E7DFC0F30894089575916591559152
:106FE8004591159011FA259035900895F9DF041B05
:106FF80010E003C0F4DF041B150B20E030E005C0EF
:10700800ECDF041B150B260B370BB8F010FC17C070
:1070180045910590E00FF11F0417100540E0240783
:10702800340758F436F404910024F101E01BF00908
:107038000994E00FF11F25903590F101099411F49E
:10704800D6F7F1CF31960EF0319650E060E070E05F
:1070580045914B3F48F089F34F3F29F04E3F11F0DF
:107068007591659155914591041B150B260B370BAE
:1070780039F318F3E7CFFA92EA92DA92CA92BA92FF
:10708800AA929A928A927A926A925A924A92BA9357
:10709800AA939A938A930895FF84EE84DD84CC841E
:1070A800BB84AA84998488847F806E805D804C80AC
:1070B800BB81AA8199818881F0E0EC0FFD1FEF0167
:1070C80008950E944338229741E050E060E070E064
:1070D8000E94D13760F440E00E94C73721F402E2F1
:1070E8006BD03FEF5FC001E267D03FE75BC0AE0106
:1070F8000E94D834C801D90143EF54E065E37FE327
:107108000E94D13768F437FBAA0FBB1FB395B69519
:10711800A795B7F908811981015010400883198390
:1071280040E050E060E87FEB43D02801390140E0BF
:1071380050E060E87FE33CD0A801B90182019301E7
:107148000E944837C801D901A801B9012FD02801E8
:1071580039010881102F110F110B212F312F0E9497
:107168000F3648E152E761E37FE320D04801590137
:1071780042E252E964ED7EE38201930117D04DEDBE
:107188005BE96AE27FE316D0A201B3010FD044E0C5
:1071980050E060E070E40ED0AC01BD0107D0A4015E
:1071A800B50108D02296ECE00C9454380C94CF36F4
:1071B8008C019D010C946E36E2EAFBE20083518358
:1071C8000FEF1FEF2FE7089501E008950E943F3861
:1071D800EF97EF976A972A873B874887598768010F
:1071E8007B0100E00B830C8302C011D21BD20AD2B0
:1071F800053251F00023C9F70B811C81EF96EF96F9
:107208006A96E0E10C9450380081053221F402D2EC
:10721800FED105E2EBCF00E00F830E830A830983DA
:107228003E0102E1600E00E0701E0FE515E2088BDA
:10723800198B06C00981002311F400810983EAD162
:10724800D9D10052B9F3035059F00850B1F30250A4
:1072580019F0035049F00CC00A8103950A83EFCF57
:107268000E8103950E83EBCF0F8103950F83E7CF34
:1072780000810A3279F4AAD1AD90BD9098D1BB2093
:107288003AF4B194A19400E0B00A0A8103950A8304
:10729800C1D114C0AA24BB244AE050E00DC02191FA
:1072A8006F0185010E941435A22EBB24A00EB11EC9
:1072B80000EDA00E0FEFB01EA0D188F30A810023C5
:1072C80011F000E00F8396D10E32F1F4A3D192D1E0
:1072D8000A3231F47BD18D909D9069D19BD117C032
:1072E800882499244AE050E088D188F421916F01DC
:1072F80084010E941435822E9924800E911E00ED7F
:10730800800E0FEF901EF0CF88248A94982C80E08E
:1073180071D10C5421F00C5131F0045039F481E052
:10732800C80E7AD103C001E0C00ED81E6BD1EAEABC
:10733800F3E00C94FA3780FB5EF44B815C81652F97
:10734800660F660B47D140835183628363834FCFB7
:107358002B813C813FD12083318349CF37D10D9197
:10736800119625D10A8B2E0103E115D1E0C02ED14B
:107378006D907D901CD1062D072921F400E7602E21
:1073880005E2702E992022F400E1802E07E2902E6B
:1073980080E090E001C00196F30101913F010023D4
:1073A80019F088159905BCF30CD1230191958195A5
:1073B8009040680E791EBBC00E81002331F0082D65
:1073C800092919F49924882483940FE715E2088B76
:1073D800198B0881003739F4F9D0ECD000E1D5D009
:1073E80000E0098330C0F1D046F40D911D912D9134
:1073F8003D91DDD0C801D90101C0DCD008810F362C
:1074080011F408E0ECCF053749F70AE0E8CFDDD002
:107418004D915D9126F46D917D91C9D005C0C7D07D
:10742800652F660F660B762FCA01DB0177234AF4B6
:107438000DE209839095A095B09581959F4FAF4F28
:10744800BF4F0AE0A2D03E0107E9600E00E0701EBF
:107458002E0107E9A0D0082F092B0A2B0B2B11F0BE
:1074680001E001C000E00D83082D092919F40D8100
:1074780000FF1FC094D0E889F989E00DF11D008153
:10748800F30102933F018BD0C801D901012B022BD4
:10749800032B81F799206AF40F81002351F0A3D0C0
:1074A80010E04501801A910A04C000E3F301029339
:1074B8003F018E0109561F4F0619170908151905AE
:1074C800A4F30E81002399F10D8100FF30C00881DB
:1074D800083711F0083549F474D0F30108810083A6
:1074E80070D000E3F301008322C00F3601F5F301E9
:1074F80000810033E1F000E302933F0118C000E986
:10750800602E05E2702E462C502EF20100810023D9
:1075180071F001E040D0F9CF0FEFC00ED01E03EBA1
:10752800602E05E2702E06EB402E05E2502E420139
:1075380086189708A814B9041CF480E090E007C0E6
:1075480052D0A818B90810E0A01AB10AC5010A81DA
:10755800002321F401C063D00197EAF709810023D1
:1075680039F055D004C053D0F30101913F015AD0EE
:107578000FEF800E901EBAF70A81002309F437CE68
:1075880001970AF434CE4BD0FBCF10E00C871D874F
:107598001E871F870895400E00E0501E08954C85F1
:1075A8005D856E857F858C019D010C948A35A0834D
:1075B800B18308958D919D91A083B183A0E0B0E03F
:1075C80008950FEF600E701E089580FBF701A081EB
:1075D800B1810895F701A081B1810D911D91A0831A
:1075E800B183F80108950981002311F001E008959D
:1075F80000E00895F60100810895F6010081005326
:107608000A300895F60101916F01088308952885CD
:107618003985089501E0C00E00E0D01E0895288540
:10762800398500E2EA85FB8509950B811C810F5F8E
:107638001F4F0B831C8308950E944B38C801D90142
:107648001A013F7740E856E968E17BE40E94E93790
:1076580038F416D0B38300E010E020E030E00DC02D
:107668003B2F0E941C360E940F360AD03383A80194
:10767800B9018C019D010E94B236E4E00C945C389B
:10768800F10100831183228308950E943F38C801C5
:10769800D901BF7741E050E060E87FE33B2F0E94CB
:1076A800D13770F440E00E94C73729F40BED1FE092
:1076B80029E43FE350C0CC24DD24EE24FF241CC081
:1076C8000BEDC02E0FE0D02E09E4E02EF72E40E09F
:1076D8007FEB082F48D02801390140E050E060E8EE
:1076E8007FE38C019D013FD0A801B901820193017C
:1076F8000E944837C801D901AC01BD018C019D0128
:107708002DD02801390144E25FEF6BE27CEB26D0F3
:1077180048E854E466EA7EE328D048E150EC6FE399
:1077280070E423D045EB1CD0480159014AEE54EBD4
:1077380066E870E48201930118D046EB11D0A801E5
:10774800B901840195010E944837AC01BD0106D0FA
:10775800A601B70108D0E0E10C9450380C94CF365C
:107768005DEF68E670E40C946E36FDDFA201B301AC
:10777800F5CF20E006D0E9F70895259102D0E9F782
:1077880008952D9301501040202F212B089580E556
:107798009AE7FC0105911491FC013296A591B491E8
:1077A800FC01349625913491422F432B19F0F901AD
:1077B800E4DF01C0DEDF06961AE78C35910748F34F
:1077C800089540E00C94E83B0E9447382897802FA2
:1077D800B32F442E40E050E060E070E00E94D137C3
:1077E80010F401E001C000E0000F400EBF7743E84D
:1077F80059EF62E27FE3082F3B2F80D076D041E03B
:107808005CEF6FE777E40E94E93788F5AE010E94E4
:10781800203B6BD0042D10E06BD0488159816A81E0
:107828007B8172D0088319832A833B83AE014C5F26
:107838005F4F2A0140E050E060E87EE35FD0A2019C
:107848000E94203B40E050E060E870E40C811D811C
:107858002E813F8153D0A801B901088119812A815D
:107868003B810E94B2360E941C36402E0CC00E94FA
:107878001C36602E3DD0A801B9018C019D0133D082
:10788800460C03E0402240FA3EF4AC01BD0100E0A2
:1078980010E020E83FE327D002E0401608F0B05897
:1078A8008C019D0129D0280139014BEF57ED6EE17C
:1078B80079E324D045E656E269E97BEB21D048E537
:1078C80054E363EA7DE31CD041EE5DE565E27FEBBE
:1078D80017D04BED5FE069EC7FE316D00DD028960A
:1078E800E8E00C9458380E94B236C801D9010895CE
:1078F80020E030E00C941A36AC01BD010C94CF3670
:1079080003D0A201B301FACF0C946E361B2F6A2F55
:10791800F901A081B181AD014F5F5F4F4083518371
:107928000C93A62FB12F0895BA93AA9324970A838C
:107938001B8389019E012A5F3F4F28833983BE013B
:10794800AE014E5F5F4F2AE83CE30E94EA3820E030
:10795800AA81BB812C932496A991B99108950E947C
:10796800433822974801590141E050E060E070E057
:107978000E94D13798F440E00E94C73729F400E00C
:1079880010E020E030E04EC001E2E2EAFBE20083D2
:1079980051830FEF1FEF2FE73FE744C0AE010E946E
:1079A800D834C801D90145EC53E062E47FE30E9472
:1079B8006E364AE151E562E17FE33BD0A801B901A7
:1079C8008C019D013BD0402E088100FF14C00A9510
:1079D8002DD0802F43EF54E065EB7FE3042D0E9408
:1079E800CF3637FB220F331F380F3695279537F9D7
:1079F800C801D9010BC01AD0842D912FD90137FBAA
:107A0800AA0FBB1FB00FB695A795B7F940E050E095
:107A180060E87EE38C019D010CD0AC01BD018401BE
:107A280095010CD02296ECE00C94543842E00C946A
:107A380004350E94CF362801390108950E9448373D
:107A4800A201B3010C946E36930424215C7AED05EF
:107A5800B72500004E6F726D610046617374200097
:107A6800466173742B00416E6C004F6E004F6E2B95
:107A780000766469200056444920002D20504C456A
:107A88004153452057414954202D2000204C6F7701
:107A9800204261747465727920212121002A2A2AE2
:107AA8004F4B212A2A2A002A4572726F7272212AA4
:107AB800002045524153494E4720454550524F4DAD
:107AC8002120002020726164696F646F6D2E6F72CF
:107AD800672020004B504F54202A2A2A4446582A0F
:107AE8002A2A2025632000466163746F7279207307
:107AF800657474696E677300202020536574746917
:107B08006E6773202020202000553D256420493DC4
:107B1800256420456D3D2564202020004D3D2564C9
:107B280020413D25642047623D25642C25642A2593
:107B380064200054582025642D25644B487A20255C
:107B4800646D4120200052582025646D5620202065
:107B5800200025642A25645F2573200020202054F6
:107B680075726E20636F696C21003C202564206D5E
:107B780056203E00436F696C20626C3F2059657344
:107B880020272B2700202020202020202020002014
:107B98002564256446256425632564762564002BC1
:107BA800253032645B205D20002D253032645B2057
:107BB8005D002B253032645B205D002020202020D2
:107BC80020202020200020464500202020202020A2
:107BD8002050502020202020202000532564256498
:107BE80046256425632564762564002564202020C5
:107BF8002020200050726F66696C652020202020AC
:107C0800202020200054623D25642E256456202023
:107C180055623D25642E25645620004261747465C2
:107C2800727920202020203C25643E002B256420EA
:107C38002020202D2E2E2E2E2E2E2E2E2B00436F62
:107C48006E74722E2020202020202020202020004A
:107C580025646D4120202020202020202020202065
:107C68002020004672657125642D2564487A20001D
:107C78004D616E75616C2D25642020202020202008
:107C880020002A46657269742000256425632D2525
:107C98006425632020200025646D41202020002DCC
:107CA8002E2E2E2E2E2E2E2B00506F7765722E2004
:107CB800202020202020202020002A2564202A257A
:107CC8006420002D2E2E2E2E2E2E2E2E2B004761B8
:107CD800696E202020202020202020202020002520
:107CE800646D562020202020200020413D2564205E
:107CF80020202020002A436F696C20626C2E2066A9
:107D08003D25642563202020200025642020202094
:107D180020004850462020202020202020202020FD
:107D2800202000466163746F7279207365747469EA
:107D38006E677352657475726E005265742E577251
:107D4800202020204E4F2059455300534C2E257398
:107D58002000566F6C756D65202020202020202083
:107D6800202000506F6C797068002564746F6E6510
:107D780020004265657073202020202020202020CC
:107D880020200025732564202D2E2E2E2E2E2E2EFB
:107D98002E2B00496E642B417520202020202020A6
:107DA80020202000257320282564292D2E2E2E2EF4
:107DB8002E2B004D6F64652C46696C7420202020A2
:107DC8002020200038363432302F303132333435E9
:107DD800363738530028253032643A253032642942
:107DE8003C253032643A253032643E200047726FB9
:107DF800756E6420626C2E4572726F722100477234
:107E08006F756E6420626C2E202D4F4B2D20002044
:107E180020202A2A2A202564202A2A2A20202020D5
:107E2800002020202020202020202020202020206A
:107E380020002B30305B200020204E6F20466572DA
:107E48007269746521202020002054616B652046EA
:107E58006572726974652120200020202020204549
:107E680072726F72212020202020002020202020E4
:107E7800204F4B2120202020202020002A2A205774
:107E880052414954204F4B21202A2A20009001308A
:107E98003132333435363738394142434445460068
:107EA800286E756C6C20706F696E7465722900306D
:107EB8003132333435363738396162636465660088
:107EC800464C4F4154533F2077726F6E6720666F60
:107ED800726D617474657220696E7374616C6C651F
:077EE8006421003F3F3F0051
:0400000300000000F9
:00000001FF
